:020000040800F2
:100000000080002055AE0008C1680008C5680008DF
:10001000C9680008CD680008D16800080000000029
:10002000000000000000000000000000D56800088B
:10003000D968000800000000DD680008E1680008D9
:10004000A5AE0008A5AE0008A5AE0008A5AE000844
:10005000A5AE0008A5AE0008A5AE0008A5AE000834
:10006000A5AE0008A5AE0008A5AE0008E56800082A
:10007000F1680008A5AE0008FD68000809690008DD
:10008000A5AE00080000000015690008A5AE000834
:10009000A5AE0008A5AE0008A5AE0008A5AE0008F4
:1000A000A5AE0008A5AE0008A5AE0008A5AE0008E4
:1000B000A5AE0008A5AE0008A5AE0008A5AE0008D4
:1000C000A5AE0008A5AE0008A5AE0008A5AE0008C4
:1000D000A5AE000821690008A5AE0008A5AE00087D
:1000E000A5AE0008A5AE0008A5AE0008A5AE0008A4
:1000F000A5AE0008A5AE0008A5AE000800000000EF
:1001000000000000A5AE000800000000A5AE000839
:10011000A5AE000800000000A5AE00082D6900088B
:10012000A5AE0008A5AE0008A5AE0008A5AE000863
:10013000A5AE00080000000000000000A5AE000809
:10014000A5AE0008A5AE00080000000000000000F9
:10015000000000000000000000000000000000009F
:10016000000000000000000000000000A5AE000834
:10017000A5AE000800000000000000000000000024
:1001800000000000A5AE0008000000000000000014
:10019000000000000000000000000000000000005F
:1001A0000000000000000000A5AE0008A5AE000899
:1001B000A5AE0008A5AE0008A5AE0008000000002E
:1001C00000000000A5AE00080000000000000000D4
:0801D000A5AE0008A5AE000871
:100200000348044B834202D0034B03B118477047A5
:10021000740600207406002000000000054806490E
:10022000091A891001EBD171491002D0034B03B1B7
:100230001847704774060020740600200000000074
:1002400010B5064C237843B9FFF7DAFF044B13B11E
:100250000448AFF300800123237010BD7406002012
:1002600000000000A8AE000808B5044B1BB104490B
:100270000448AFF30080BDE80840CFE7000000006D
:1002800078060020A8AE000870B50D4E0D4D761B07
:10029000B61006D00024013455F8043B9847A64216
:1002A000F9D1094E094D761B0AF0FEFDB61006D0B5
:1002B0000024013455F8043B9847A642F9D170BD9B
:1002C00058B2000858B200085CB2000858B20008E2
:1002D000024B0146186800F043B900BF000000203F
:1002E000024B0146186800F0E7B800BF000000208C
:1002F000844641EA000313F003036DD1403A41D331
:1003000051F8043B40F8043B51F8043B40F8043BEF
:1003100051F8043B40F8043B51F8043B40F8043BDF
:1003200051F8043B40F8043B51F8043B40F8043BCF
:1003300051F8043B40F8043B51F8043B40F8043BBF
:1003400051F8043B40F8043B51F8043B40F8043BAF
:1003500051F8043B40F8043B51F8043B40F8043B9F
:1003600051F8043B40F8043B51F8043B40F8043B8F
:1003700051F8043B40F8043B51F8043B40F8043B7F
:10038000403ABDD2303211D351F8043B40F8043B1F
:1003900051F8043B40F8043B51F8043B40F8043B5F
:1003A00051F8043B40F8043B103AEDD20C3205D32F
:1003B00051F8043B40F8043B043AF9D2043208D027
:1003C000D2071CBF11F8013B00F8013B01D30B8899
:1003D00003806046704700BF082A13D38B078DD077
:1003E00010F003038AD0C3F10403D21ADB071CBF49
:1003F00011F8013B00F8013B80D331F8023B20F8B3
:10040000023B7BE7043AD9D3013A11F8013B00F8EB
:10041000013BF9D20B7803704B7843708B78837073
:1004200060467047F0B4860743D0541E002A3ED081
:10043000CAB2034602E014F1FF3438D303F8012BAB
:100440009D07F8D1032C2BD9CDB245EA05250F2CF9
:1004500045EA054516D9A4F110073F0903F1200626
:1004600006EB071603F1100242E9045542E9025572
:100470001032B242F8D104F00F040137032C03EB21
:1004800007130DD91E462246043A032A46F8045B98
:10049000FAD8221F22F003020432134404F00304AA
:1004A0002CB1C9B21C4403F8011B9C42FBD1F0BC27
:1004B000704714460346C5E779B338B551F8043C94
:1004C0000C1F002BB8BFE418054600F087F9234B3A
:1004D0001A682AB1A2420DD921686018824230D030
:1004E000626028461C60BDE8384000F079B9A3423C
:1004F00003D81A465368002BF9D111685018A0424E
:1005000013D00BD821686018834220D063605460F8
:100510002846BDE8384000F063B970470C232B60D3
:100520002846BDE8384000F05BB920680144501807
:1005300083421160ECD1D3E90003014453601160A0
:10054000E6E7D2E90002014462602160C9E7D3E92D
:1005500000030144636021605460D9E790060020E5
:10056000F8B5CD1C25F0030508350C2D38BF0C253A
:10057000002D06463ADBA94238D82A4F00F02EF962
:100580003A6852B113685B1B04D433E023685B1BE9
:1005900025D522465468002CF8D1796800293BD033
:1005A0002946304600F040F8431C2AD0C41C24F0F1
:1005B0000304A04205D0211A304600F035F801307E
:1005C0001FD02560304600F00BF904F10B0020F03D
:1005D0000700231DC31A01D05A42E250F8BD0B2B6D
:1005E0000BD8A24215D063685360EBE70C2333604D
:1005F0000020F8BD0B2B0BD9144623601C4425604A
:10060000E0E70C233046336000F0EAF80020F8BD44
:1006100054683C601446D5E7304600F005F8786031
:10062000BEE700BF9006002038B5074C0023054602
:100630000846236003F08AF8431C00D038BD2368C5
:10064000002BFBD02B6038BD447400200CB470B577
:100650009CB020AC0B4E54F8042B0291234606911B
:100660006FF0004502A901940795CDE9045600F00A
:1006700093F9029B00221A701CB0BDE8704002B0D2
:10068000704700BF0802FFFF0EB430B59CB01FAB2F
:100690000C4C0D4D53F8042B019301460291069129
:1006A000206802A96FF000440794CDE9044500F0EA
:1006B00073F9029B00221A701CB0BDE8304003B0F1
:1006C000704700BF000000200802FFFF000000008C
:1006D000000000000000000000000000000000001A
:1006E000000000000000000000000000000000000A
:1006F00000000000000000000000000000000000FA
:1007000090F800F06DE9024520F007016FF0000C51
:1007100010F0070491F820F040F049804FF00004F9
:100720006FF00700D1E9002391F840F000F10800D4
:1007300082FA4CF2A4FA8CF283FA4CF3A2FA8CF30C
:100740004BBBD1E9022382FA4CF200F10800A4FA73
:100750008CF283FA4CF3A2FA8CF3E3B9D1E90423C7
:1007600082FA4CF200F10800A4FA8CF283FA4CF3FE
:10077000A2FA8CF37BB9D1E9062301F1200182FAB8
:100780004CF200F10800A4FA8CF283FA4CF3A2FABE
:100790008CF3002BC6D0002A04BF04301A4612BACC
:1007A000B2FA82F2FDE8024500EBD2007047D1E9CF
:1007B000002304F00305C4F100004FEAC50514F05E
:1007C000040F91F840F00CFA05F562EA05021CBF2F
:1007D00063EA050362464FF00004A9E7704700BFD3
:1007E000704700BF2DE9F0478E681D46AE420C46AB
:1007F0000B68174627D88046888910F4906F31D04F
:10080000D1E9041606EB4606A3EB010906EBD67602
:100810006B1C76104B44B342324684BF1E463246B0
:10082000430521D511464046FFF79AFE824678B32C
:100830004A462169FFF75CFDA38923F4906343F0E6
:100840008003A38115E02E4618462A46394600F05B
:1008500007FCA2682368961B2B44A6602360002037
:10086000BDE8F0873546EFE7404600F05DFC824684
:1008700050B1A6EB09020AEB09036661C4F810A0A7
:100880002360A2602E46DFE721694046FFF714FE91
:100890000C23C8F80030A38943F04003A3814FF034
:1008A000FF30DDE72DE9F04F936883B09046002BD1
:1008B0006CD017688D6882460C460868083742E09D
:1008C000A38913F4906F2DD0D4E9041505EB4505E9
:1008D000A0EB010B05EBD575701C6D105844A842B8
:1008E0002A4684BF05462A465B0536D51146504642
:1008F000FFF736FE00283AD05A4621690190FFF7EB
:10090000F7FCA289019B22F4906242F08002A2814E
:10091000A5EB0B0203EB0B00656123612060A26075
:100920003546B3465A46494600F09AFBD8F8083097
:10093000A2682068551B58449E1BA5602060C8F81B
:1009400008601EB3083757E90296AB46002EF9D06F
:10095000AE42B5D23546B346E4E7504600F0E4FB7C
:1009600003460028D4D121695046FFF7A5FD0C238A
:10097000CAF80030A389002243F040034FF0FF3053
:10098000A381C8E9012203B0BDE8F08F0020C8F8B8
:10099000040003B0BDE8F08F2DE9F04F14468A89BA
:1009A0009FB015068946029003D50A69002A00F017
:1009B0001281059330238DF832302378904E002138
:1009C00020220B918DF831200127002B00F092801E
:1009D000252B254603D118E0252B00F0BD8015F806
:1009E000013F002BF8D1B5EB040B00F083802246C9
:1009F0005B4649460298FFF7F5FE01307AD00B9B23
:100A00002A785B440B93002A74D000234FF0FF3206
:100A100001350693CDE908338DF85B301C930792BE
:100A200005E0069A07FA03F3134355460693AA46D0
:100A300005221AF8011B304600F0C2FAD346831B88
:100A40000028EED1069BD90644BF20228DF85B20FA
:100A500029781A0744BF2B228DF85B202A2953D00E
:100A6000A1F13003092B00F2AB80099A02E0554650
:100A70000AF1010A9AF8001002EB820203EB42022B
:100A8000A1F13003092BD346F1D905F1020A0992ED
:100A90002E2945D05B4C0322204600F091FA002815
:100AA00057D0001B069A402404FA00F00243069235
:100AB0000AF101049AF8001053488DF8301006220C
:100AC00000F07EFA002859D0504B002B49D005ABDE
:100AD00000934A464E4B029806A9AFF30080804629
:100AE000B8F1FF3F06D00B9B43440B932378002BB8
:100AF0007FF46EAFB9F80C305B0654BF0B984FF023
:100B0000FF301FB0BDE8F08F059A1168043200294C
:100B100005922DDB099169782E2905F1020AB9D1D8
:100B20009BF801102A2933D1059B9BF802101A6803
:100B300007920433002A05930BF102000BF1030A1C
:100B400040DB304C83460322204600F039FA00286F
:100B5000A7D15446DA46ADE7B5EB040B3FF455AFE9
:100B600045E7059B073323F0070308330593BAE7EE
:100B7000494243F0020309910693CCE705AB009389
:100B80004A46234B029806A900F0D2F88046A7E710
:100B9000A1F1300000220928079201D917E0DA46B6
:100BA0009AF8011002EB820200EB4202A1F1300040
:100BB00009280AF1010BF2D90AF1020A079269E742
:100BC000AB4665E74FF0FF328346079262E7D346B4
:100BD0000AF1010A5EE740210393FFF7C1FC039B82
:100BE000C9F80000C9F8100018B14022C9F8142053
:100BF000DFE6029A0C2313604FF0FF3081E700BF5D
:100C000008B2000810B2000814B20008000000008A
:100C1000E50700082DE9F0470C4691460A69896806
:100C2000DDF820808A42B8BF0A46C9F8002094F84F
:100C3000431006461F4611B10132C9F8002023684F
:100C400099065FD5D9F800200232C9F80020236840
:100C500013F0060F19461DD1E1688A1A002AD8BF81
:100C6000194617DD04F1190A002505E0E368D9F8F3
:100C700000209B1AAB420CDD012352463946304618
:100C8000C047013005F10105F0D14FF0FF30BDE85C
:100C9000F087216894F84330003318BF01238A0697
:100CA0000AD5E1185A1C302081F84300224494F8F8
:100CB000451082F84310023304F1430239463046AE
:100CC000C0470130E1D02368D9F80050216903F012
:100CD0000603042BD4E902201AD08A421FDD4FF00C
:100CE0000009521A91441A34002501E04D4516D0EE
:100CF0000123224639463046C047013005F101053F
:100D0000F4D1C2E713F0060F0CD1D9F80020A3E705
:100D1000401B8A4220EAE079E3DC0028E3DC002083
:100D2000BDE8F08794F84330003318BF0123C3E7D0
:100D30002DE9F0430C46097E85B06E2906460C9DD0
:100D40001746984604F1430C4AD00FD8632900F0A7
:100D5000FF8000F2BF8000294ED0582940F0E1808A
:100D600084F845102268DFF844E212E0732900F0AD
:100D7000C6807AD86F2900F0DB80702940F0D180DE
:100D8000206840F0200222607823DFF824E284F813
:100D900045302B68191D1B682960150602D45006C2
:100DA00048BF9BB2D10744BF42F020022260002B13
:100DB0006DD1D4E9001284F84330002A21F02003D9
:100DC0002360A2607EDB21F0240121601021002A33
:100DD00079D1654608294ED0ACEB050323610EE0BE
:100DE0002B6822686169181D286015061B6802D4EB
:100DF000500600F1C7801960002365462361CDF8D5
:100E000000803B4603AA21463046FFF703FF01302E
:100E100020D02A46236939463046C047013019D0D0
:100E200022680398E368920719D51A1A002A16DD7A
:100E300004F11909002504E0E36803981A1AAA428C
:100E40000DDD01234A4639463046C047013005F1E1
:100E50000105F1D14FF0FF3005B0BDE8F0839842B5
:100E6000B8BF184605B0BDE8F083752960D0782971
:100E700057D1226888E72368DB07ADD5626823690C
:100E80009A42A9DC302305F8013C013DA4E710217A
:100E9000002284F843206268A260002A2CDB2068CC
:100EA00020F004002060002B91D06546B3FBF1F2E6
:100EB00001FB123013461EF8002005F8012D002B0F
:100EC000F4D187E710219EF8003084F8423004F115
:100ED00042057FE7642901D0692922D120682B6867
:100EE000010603F1040245D51B682A60002B4BDB89
:100EF000DFF8B8E00A21CEE7002BD6D1E3E72B6874
:100F00006268191D29601D680021284600F058F804
:100F1000002848D0401B60602061002384F84330E3
:100F20006DE7012384F84210236104F14205F4E7E0
:100F300020682B6810F0800F03F1040213D01B68A7
:100F40002A606F290CBF08210A21DFF860E09FE7C3
:100F50002B681A68191D0123296084F84220236137
:100F600004F14205D9E7400653BF1B682A601B887D
:100F70002A60E6E7410653BF1B682A60B3F90030D8
:100F80002A60B3E7198037E76268A2602D21002A42
:100F900084F84310C3F10003DFF810E04FF00A01BA
:100FA000BFF67EAF81E76068B6E700BF1CB20008FD
:100FB00030B2000800000000000000000000000047
:100FC00001F0FF01102A2BDB10F0070F08D010F8FA
:100FD000013B013A8B422DD010F0070F42B3F6D1FE
:100FE000F0B441EA012141EA014122F007047FF017
:100FF00000070023F0E80256083C85EA010586EA6E
:10100000010685FA47F5A3FA87F586FA47F6A5FAA9
:1010100087F68EB9EED1F0BC01F0FF0102F00702B5
:1010200032B110F8013B013A83EA010313B1F8D160
:101030000020704701387047002D06BF3546033841
:10104000073815F0010F07D1013015F4807F02BF7A
:10105000013015F4C03F0130F0BC0138704700BFCB
:101060008842F0B40DD98B1883420AD9841832B162
:10107000224613F8014D02F8014D9942F9D1F0BC16
:1010800070470F2A49D940EA01039B0747D1A2F1D3
:1010900010031B0901F1200707EB031701F11004EE
:1010A00000F1100554F8106C45F8106C54F80C6CF5
:1010B00045F80C6C54F8086C45F8086C54F8046C4E
:1010C00045F8046C1034BC4205F11005EAD1013337
:1010D00002F00F051B01032D1944034421D91F1FE2
:1010E0000E462C46043C56F804CB47F804CF032C9C
:1010F000F8D82C1F24F0030404342344214402F0C4
:101100000302002ABBD0013B0A4411F8014B03F84B
:10111000014F9142F9D1F0BC70470346F1E7034615
:10112000F1E72A46EDE700BFE1B1F8B51446E2B1B8
:1011300006460D4600F01EF8A04202D32F46384660
:10114000F8BD21463046FFF70BFA07460028F6D0D7
:1011500022462946FFF7CCF830462946FFF7ACF97E
:101160003846F8BD1146FFF7FBB9FFF7A5F927464A
:10117000E5E700BF51F8043C181F002BBCBF0B581B
:10118000C01870470000000000B551EC100B2C4A4D
:1011900021F00043934285B020DD2A4A934209DDC5
:1011A00010EE102A0B4602F0E3FA41EC100B05B0EA
:1011B0005DF804FB684600F0FBFF00F00300012827
:1011C00017D002282FD028B301209DED021B9DEDE2
:1011D000000B02F031F851EC100BE6E79FED161B07
:1011E00001F0DAFA51EC100B41EC100B05B05DF890
:1011F00004FB9DED021B9DED000B02F01DF853EC6E
:10120000102B10EE100A03F1004141EC100B05B059
:101210005DF804FB9DED021B9DED000B01F0BCFA97
:1012200051EC100BC1E79DED021B9DED000B01F091
:10123000B3FAE4E7AFF30080000000000000000014
:10124000FB21E93FFFFFEF7F00B551EC100B2C4A6B
:1012500021F00043934285B027DD2A4A934209DDFD
:1012600010EE102A0B4602F083FA41EC100B05B089
:101270005DF804FB684600F09BFF00F003000128C6
:101280001FD0022830D028B39DED021B9DED000B2E
:1012900001F082FA53EC102B10EE100A03F100411A
:1012A00041EC100B05B05DF804FB00209FED121B14
:1012B00001F0C2FF51EC100B41EC100B05B05DF8D2
:1012C00004FB9DED021B9DED000B01F065FA51EC56
:1012D000100BCAE701209DED021B9DED000B01F0F4
:1012E000ABFF51EC100BC0E701209DED021B9DED03
:1012F000000B01F0A1FFCDE700000000000000009E
:10130000FB21E93FFFFFEF7F2DE9F04F2DED028B31
:10131000DFF824A38BB057EC106B55EC114B00F0A9
:10132000EBF99AF90080B0EE408AF0EE608AB8F1ED
:10133000FF3F33D022462B462046294602F06AFE64
:10134000834658BB32463B463046394602F062FE81
:101350008146002866D1304639460022002302F03B
:1013600027FE20B3002200232046294602F020FE5B
:10137000834600287DD09FEDA67B0122AA4BCDF8A5
:1013800020900092CDE90267CDE904458DED067B02
:101390000193B8F1000F5ED09FED9F8BB0EE480A2D
:1013A000F0EE680A0BB0BDEC028BBDE8F08FB0EE3A
:1013B000480AF0EE680A02F013F88046002800F0B0
:1013C00082804FF000084FF0000951EC180B4246A4
:1013D0004B4602F0EDFD0028E0D047EC106B01F029
:1013E000FFFF0028DAD045EC104B01F0F9FF002890
:1013F000D4D09AF900308C4A019204210022022BA9
:10140000CDE90267CDE90445CDE90689009108924E
:1014100003D0684602F074F810BB03F009F82223E9
:1014200003601DE0002200232046294602F0C0FD93
:101430000028B3D09FED788B01227B4BCDF820B0F4
:10144000B8F1020F0092CDE90267CDE904458DEDB8
:10145000068B0193A2D0684602F052F8002878D09B
:10146000089B1BB102F0E4FF089B03609DED068B17
:1014700094E745EC104B01F0B3FF00288ED000221A
:1014800000232046294602F09DFD002886D0664AAA
:101490009AF90030CDF820B00121CDE90267CDE9FD
:1014A0000445CDE90012002B58D060490020022BE2
:1014B000CDE9060156D102F0BBFF21230360089B52
:1014C000002BD3D0CEE747EC106B01F089FF00284A
:1014D0003FF477AF45EC104B01F082FF00283FF45A
:1014E00070AF53EC182B18EE100A194602F092FD5B
:1014F0009AF9009000286FD10323DFF82CC10890DF
:101500002946204600930022494BCDF804C0CDE97E
:101510000445CDE9026702F0E3FA04460D46B9F14D
:10152000000F25D1DFF814914FF06048002200230E
:1015300030463946CDE9068902F044FD38BB68469D
:1015400001F0DEFF0028BAD102F072FF222303600F
:10155000B5E702F06DFF2123036081E79FED2C7B4F
:101560008DED067B684601F0CBFF0028A7D1A2E7EE
:101570009FED2B7B00220023304639468DED067B04
:1015800002F020FDB0B9B9F1020FDDD0D7E745EC8C
:10159000104B01F0C1FF22462B4651EC100B02F01C
:1015A00007FDB0B9234B9AF900904FF06042CDE9A6
:1015B0000623E8E745EC104B01F0AEFF22462B4630
:1015C00051EC100B02F0F4FC18B9184B0022CDE9D5
:1015D00006239AF90090D6E70122134BCDF820801C
:1015E0000092CDE90267CDE904450193B9F1000FFE
:1015F000B4D0002200231046194602F09BFBB9F13B
:10160000020FCDE906013FF456AFABE7AFF3008020
:101610000000000000000000000000000000F03F9B
:10162000000000000000F07F44B200080000F0FF5E
:101630000000E03FFFFFEFC764000020FFFFEF471F
:101640002DE9F0432DED028B8BB055EC104B00F0E3
:10165000D9FF274BB0EE408AF0EE608A93F9006024
:10166000731C12D022462B462046294602F0D2FC9B
:10167000074650B94FF000084FF0000920462946B0
:1016800042464B4602F09EFC40B9B0EE480AF0EEEE
:10169000680A0BB0BDEC028BBDE8F0830122154B4C
:1016A00008970092CDE90445CDE90245019396B132
:1016B00042464B464046494602F03CFB022ECDE9ED
:1016C00006010AD102F0B4FE21230360089B53B93E
:1016D0009DED068BD9E7CDE90689684601F010FF3C
:1016E0000028F3D1EEE702F0A3FE089B0360EFE7CA
:1016F0006400002048B200082DE9F04F51EC110BB6
:1017000021F0004555EA000393B010D059EC108B3E
:101710006D4B29F000449C424E4610EE10AA0DDDA0
:1017200004F1404404F5801454EA0A0356D1674991
:10173000002041EC100B13B0BDE8F08F0F4611EE06
:1017400010CA48D09D42EBDC5F4B9D425FD0002E1B
:10175000CDE900015FDB4FF0000BBCF1000F0ED1B3
:10176000594B9D4243D0594B9D4200F08C80B7F1BC
:10177000804F00F09E80564B9F4200F0B88349ECAA
:10178000108B01F023FE51EC100BBAF1000F06D1C3
:10179000002C5AD04D4B26F040429A4255D0F60FBD
:1017A00006F1FF3A5BEA0A0373D04A4B9D4240F3CD
:1017B000998003F104739D4240F33884464B9C4268
:1017C00072DD002F72DD3EA3D3E9002310461946D7
:1017D00002F086F9ADE7B8F1000F05D03F4813B02D
:1017E000BDE8F04F01F090BEA542F7DCACE704F194
:1017F000404303F5801353EA0A0398D0364B9C42CA
:1018000040F37F83002F51DBDDE9000191E7BCF15C
:10181000000F9CD084E7324B9D4231DCA3F154731E
:101820009D4298DD2B15A3F2FF33142B40F3A183C7
:10183000C3F134032CFA03F202FA03F363458AD1AD
:1018400002F00102C2F1020B87E7002F05DA02461F
:101850000B4600201D4902F06DFA002EBFF669AF5D
:1018600004F1404404F5801454EA0B0300F03A8478
:10187000BBF1010F7FF45DAF01F10043194658E75A
:101880004FF0020B69E7002FC0F2448340464946FF
:101890004FE742464B461046194601F069FF0246A3
:1018A0000B4602F047FA44E7002F8CDB00200021B2
:1018B0003FE742464B464046494602F011F938E7B9
:1018C0009C7500883CE4377E0000F07F0000F03F0C
:1018D0000000E03F0000E041FFFFEF3F2CB20008B6
:1018E000FFFF3F43B4F5801F80F260830022D04B9E
:1018F00002F0F6F86FF034060C462315CD4AC4F317
:101900001304A3F2FF3344F07F559E1994420D96C1
:1019100045F4401540F33D83C74B9C4240F301849E
:101920009FEDAD7B8DED087B8DED107B9FEDAC7B4E
:101930008DED067B01360D96A5F580154FF000085C
:10194000DDE906232946064601F012FFDDE90623FC
:10195000CDE90A013046294601F00CFF02460B464C
:101960000020B64902F0E6F903460C46CDE90E34F4
:1019700002460B46DDE90A0102F0B2F86B1043F0B3
:10198000005303F500230A462F46014603EB0805E2
:101990000023CDE902120293DDE902890024CDE99A
:1019A00004122B4622464046494602F099F8024668
:1019B0000B46DDE90A0101F0DBFEDDE90623CDE996
:1019C0000A012046294601F0D3FE02460B46304666
:1019D000394601F0CDFE42464B4602F081F8024600
:1019E0000B46DDE90A0101F0C3FEDDE90E2302F03A
:1019F00077F8DDE90445CDE9060122462B4620466D
:101A0000294602F06DF878A3D3E9002304460D4679
:101A100002F066F876A3D3E9002301F0ABFE22467C
:101A20002B4602F05DF874A3D3E9002301F0A2FE77
:101A300022462B4602F054F871A3D3E9002301F0AB
:101A400099FE22462B4602F04BF86FA3D3E9002300
:101A500001F090FE22462B4602F042F86CA3D3E937
:101A6000002301F087FE224606460F462B462046FD
:101A7000294602F035F802460B463046394602F058
:101A80002FF8424604460D464B46DDE9040101F0BD
:101A900071FEDDE9062302F023F822462B4601F011
:101AA00069FE424606460F464B464046494602F00E
:101AB00017F80022624BCDE90A0101F05BFE3246C5
:101AC0003B4601F057FE02980D46044622462B463F
:101AD0004046494602F004F8002280468946584BA9
:101AE0002046294601F044FEDDE90A2301F040FECC
:101AF00002460B463046394601F03AFEDDE9042342
:101B000001F0EEFF224606460F462B46DDE90601B0
:101B100001F0E6FF02460B463046394601F02AFE48
:101B200006460F4602460B464046494601F022FE55
:101B3000029839A3D3E9002304460D4601F0D0FFF3
:101B40004246CDE904014B462046294601F010FEED
:101B500002460B463046394601F00AFE30A3D3E96F
:101B6000002301F0BDFF30A3D3E9002306460F4652
:101B70002046294601F0B4FF02460B46304639465E
:101B800001F0F8FDDDE9102301F0F4FD06460D98A3
:101B90000F4601F03BFF3246804689463B46DDE971
:101BA000040101F0E7FDDDE9082301F0E3FD424611
:101BB0004B4601F0DFFD029842464B4604460D4677
:101BC00001F0D6FDDDE9082301F0D2FDDDE90423B3
:101BD00038E000BFAFF3008000000000000000000C
:101BE000000000000000F03FEF4E454A287ECA3F4B
:101BF00065DBC9934A86CD3F01411DA96074D13F81
:101C00004D268F515555D53FFFAB6FDBB66DDB3F92
:101C1000033333333333E33F000000E009C7EE3FC3
:101C2000FD033ADC09C7EE3FF5015B14E02F3EBE31
:101C3000000040438E98030079B60B000000F03F8F
:101C40000000084001F094FD0B460246394630463C
:101C500001F08EFD0BF1FF3353EA0A03CDE90401D5
:101C600000F05F819FEDD27B8DED027BDDE900AB63
:101C7000002356465F46CDE900670093DDE9006723
:101C8000504632463B46594601F072FD22462B46ED
:101C900001F026FF5246804689465B46DDE9040195
:101CA00001F01EFF02460B464046494601F062FD28
:101CB0003246804689463B4620462946CDE904897E
:101CC00001F00EFF0B46024606460F4640464946C7
:101CD00001F050FDD04B994204460D468A4640F330
:101CE000258101F13F4303F5E003034340F0FE810A
:101CF000B1A3D3E90023DDE9040101F03BFD324645
:101D0000804689463B462046294601F031FD024681
:101D10000B464046494602F073F9002840F0E68140
:101D2000A8464FEA2853A3F2FE324FF48013134122
:101D30005344C3F30A52B94DA2F2FF321541C3F323
:101D4000130423EA05010020C2F1140B44F48014AB
:101D5000BAF1000F02460B4644FA0BFB30463946F7
:101D6000B8BFCBF1000B01F003FD06460F4632462B
:101D7000DDE904013B4601F0FDFC4FEA0B5A0D463C
:101D800000248FA3D3E900232046294601F0A8FEB2
:101D90003246804689463B462046294601F0E8FC0B
:101DA00002460B46DDE9040101F0E2FC86A3D3E91B
:101DB000002301F095FE86A3D3E9002306460F46D3
:101DC0002046294601F08CFE02460B463046394635
:101DD00001F0D0FC06460F4602460B4640464946F7
:101DE00001F0C8FC42464B4604460D4601F0C0FCDB
:101DF00002460B463046394601F0BAFC2246804680
:101E000089462B462046294601F06AFE72A3D3E993
:101E1000002306460F4601F063FE71A3D3E90023B9
:101E200001F0A6FC32463B4601F05AFE6EA3D3E910
:101E3000002301F09FFC32463B4601F051FE6CA3AB
:101E4000D3E9002301F094FC32463B4601F048FE02
:101E500069A3D3E9002301F08DFC32463B4601F033
:101E60003FFE02460B462046294601F081FC06460D
:101E70000F4602460B462046294601F031FE00225D
:101E8000CDE900014FF080433046394601F070FC47
:101E900002460B46DDE9000101F04CFF42460646D2
:101EA0000F464B462046294601F01AFE42464B4655
:101EB00001F060FC02460B463046394601F058FC02
:101EC00022462B4601F054FC02460B4600205449A2
:101ED00001F04EFC8A44BAF5801F02460B46C0F260
:101EE00030815146DDE9022301F0FAFD21E4002EA4
:101EF000FFF645AC49EC108B13B0BDE8F04F00F095
:101F000081BB002FBFF6D2ACDDE90034184604F1E6
:101F100000410EE442464B460020414901F00AFFD1
:101F200007E49FED377B8DED027B9FE63D4B21F073
:101F30000048984540F3E8803B4B0B4403430AD1EB
:101F400032463B4601F014FCDDE9042302F04EF872
:101F500000283FF4E6AEDDE902012BA3D3E900231C
:101F600001F0BEFD28A3D3E9002301F0B9FDFFF77E
:101F7000E0BBBCF1000F40F0D080C3F1140345FA80
:101F800003F202FA03F3AB4200F0E380E346FFF70B
:101F9000EABB9FED1F7B8DED087B8DED107B9FEDE8
:101FA000047B4FF000088DED067BC9E40026A4E415
:101FB000000000000000F03FFE822B654715973CB3
:101FC00000000000432EE63FEF39FAFE422EE63FC6
:101FD000396CA80C615C20BED0A4BE726937663E25
:101FE000F16BD2C541BDBB3E2CDE25AF6A56113F19
:101FF00093BDBE166CC1663F3E5555555555C53F00
:10200000000000000000F0BF59F3F8C21F6EA501E8
:102010000000000000000000FFFF8F40FFFF0F00E6
:102020000000F03FFFCB904000346F3F5C4B9C4280
:102030007FF73AAC5B4B9C423FF7C3AB0022594B56
:1020400001F096FB46A3D3E9002304460D4601F0B8
:1020500047FD45A3D3E9002380468946204629460B
:1020600001F03EFD0022CDE902014F4B20462946FA
:1020700001F036FD02460B463DA1D1E9000101F019
:1020800077FB22462B4601F02BFD02460B46002033
:10209000464901F06DFB224606460F462B46204678
:1020A000294601F01DFD02460B463046394601F037
:1020B00017FD31A3D3E9002301F012FD02460B46C0
:1020C000DDE9020101F054FB02460B4606460F46CD
:1020D0004046494601F04EFB002004460D4642466C
:1020E0004B46AFE502460B46FFF7D5BBDDE90201E3
:1020F00023A3D3E9002301F0F3FC21A3D3E90023B8
:1021000001F0EEFCFFF715BB284B98453FF709AEF1
:10211000DDE900239246934632E64FF0000BFFF7CD
:102120002EBB9FED197B8DED087B9FED197B8DED0F
:10213000107B9FED197B4FF480288DED067BFFF718
:10214000FFBB584643EC102B01F06EFA51EC100B1C
:10215000C8E602F00102C2F1020BFFF704BB00BFA8
:10216000000000604715F73F44DF5DF80BAE543EBA
:10217000555555555555D53FFE822B654715F73FAB
:102180009C7500883CE4377E0000004003B8E23FC5
:1021900006D0CF43EBFD4C3E000000000000F83FAE
:1021A000FEFFEF3F0000F03F0000D03F0000E03FA7
:1021B0002DE9F04753EC102BBF4923F000478F4225
:1021C00090B040F39380BD498F421C46824629DC83
:1021D000002C194610EE100AADA3D3E9002340F3FA
:1021E000908001F0C5FAB64B9F4204460D4600F0C0
:1021F0007381A9A3D3E9002301F0BAFA02460B4682
:10220000CAE900232046294601F0B2FAA2A3D3E985
:10221000002301F0ADFA0125CAE90201284610B0F9
:10222000BDE8F087A7498F4240F38A80A6498F42D4
:1022300000F320813D15A5F2164510EE100AA7EB1C
:10224000055116460F4601F0FBFE01F0DFFB80460C
:10225000894642464B4630463946CDE90A8901F067
:1022600087FA0022994B01F03BFC8946804601F039
:10227000E7FE01F0CBFB06460F4632463B464046A2
:102280004946CDE90C6701F073FA00228F4B01F04B
:1022900027FC00220023CDE90E0101F089FE002871
:1022A00000F06581002330463946002201F080FEAF
:1022B000002814BF01230223854A019202212A46E5
:1022C00000910AA8514600F0ABFB002C054614DA39
:1022D000DAF80420DAF80C3002F1004203F100438E
:1022E0004542CAF80420CAF80C3006E080ED000B25
:1022F00000250024C0E902450025284610B0BDE8AD
:10230000F08701F037FA6E4B9F4204460D4600F00D
:10231000108161A3D3E9002301F02CFA02460B4699
:10232000CAE900232946204601F022FA5AA3D3E93C
:10233000002301F01FFA4FF0FF35CAE90201DCE784
:1023400001F044F859EC108B10EE100A54A3D3E9B5
:102350000023494601F0C4FB00225E4B01F00AFA5B
:1023600001F06EFE054601F051FB49A3D3E90023BD
:10237000CDE9060101F0B4FB02460B464046494652
:1023800001F0F6F944A3D3E9002380468946DDE94C
:102390000601CDE9028901F0A3FB1F2D02460B4681
:1023A000CDE9042340F3B580DDE90423DDE9020132
:1023B00001F0DEF9804689463F15C9F30A53FB1A3E
:1023C000102B40F3B38038A3D3E90023DDE90601E5
:1023D00001F086FB8046894602460B46DDE9020194
:1023E00001F0C6F902460B46DDE90201CDE90823FA
:1023F00001F0BEF942464B4601F0BAF92CA3D3E9ED
:10240000002380468946DDE9060101F069FB42466A
:102410004B4601F0ADF90B46CDE904010246DDE97A
:10242000080101F0A5F9C1F30A53FF1A312F8046C4
:10243000894600F39E809DED087BCAE900898DEDF9
:10244000027B42464B46DDE9020101F091F9DDE9EC
:10245000042301F08DF9002CCAE90201BFF64DAF4B
:1024600009F1004401F100436D42CAE90084CAE960
:10247000020342E710EE100A194601F079F900252F
:10248000CAE90201CAE9000137E700BFAFF30080E3
:1024900000004054FB21F93F3163621A61B4D03D22
:1024A00083C8C96D305FE43F0000601A61B4D03D5D
:1024B0007370032E8A19A33BFB21E93F7BD90240AD
:1024C000FB21F93FFB213941FFFFEF7F0000704105
:1024D00040AF00080000E03F41A3D3E9002301F032
:1024E00047F941A3D3E900230D46044601F040F922
:1024F00002460B46CAE900232946204601F038F976
:1025000039A3D3E9002301F033F90125CAE9020117
:10251000F3E64046494601F02BF9394B6A1E8046E6
:1025200053F82230BB4289463FF446AFCAE90089DE
:1025300087E72BA3D3E9002301F01CF92AA3D3E9F1
:1025400000230D46044601F015F902460B46CAE980
:1025500000232946204601F00BF923A3D3E90023E9
:1025600001F008F94FF0FF35CAE90201C5E603237F
:10257000A2E61FA3D3E90023DDE9060101F0B0FACA
:1025800006460F4602460B46DDE9080101F0F0F869
:102590008046894602460B46DDE90801CDE90289FD
:1025A00001F0E6F832463B4601F0E2F812A3D3E927
:1025B000002306460F46DDE9060101F091FA324696
:1025C0003B4601F0D5F802460B4640464946CDE968
:1025D000042301F0CDF880468946A7E7AFF30080D9
:1025E0000000601A61B4D03D7370032E8A19A33BBA
:1025F0000000002E8A19A33BC14920259A837B390C
:10260000C0AE00082DE9F041624A57EC106BBA43A6
:1026100000F09580002F3B4610EE101A344654DD32
:102620003F1500F0AF80C3F31303A7F2FF3743F465
:102630008013E20FF90702EB43034FEA440503D589
:10264000ED0F05EB4303A50000267F10B4461622CC
:102650004FF400110CEB010098424FEAD5744FEA99
:10266000450503DC1B1A00EB010C0E44013A04EB98
:1026700043034FEA5101EDD11046964620244FF016
:10268000004209E052D05B00013C03EBD5734FEAF6
:1026900052024FEA450536D0634502EB0E01F1DDEB
:1026A000002901EB020E0ADBE046A3EB0C03A94272
:1026B00088BF03F1FF336D1A1044C446E3E7BEF14F
:1026C000000FF1DB0CF10108EFE727F00042324385
:1026D0002AD0002F49D1CA0A153B4905002AFAD051
:1026E00012F4801001D050E020465200D50200F1D3
:1026F0000104F9D5C4F1200501FA04F4E9401F1AD8
:1027000041EA02038FE72B4329D144087110F307F4
:1027100001F17F5101F5001148BF44F0004401EB85
:102720000753224643EC102BBDE8F081A942AAD8FA
:10273000002901EB020EC2DB98460023BBE710EE36
:10274000102A3B4610EE100A394601F0C9F932460C
:102750003B4601F00FF841EC100BBDE8F081421C44
:1027600016BF421C01365408D0E710EE102A30463E
:10277000394600F0FDFF02460B4601F0DBFA41EC62
:10278000100BD1E71A463B46AAE70C4620254FF02E
:10279000FF30B3E70000F07F2DE9F04F57EC106BEE
:1027A0002DED028BB0EE418AF0EE618A27F00049F0
:1027B000B9F1795F83B072DA10EE100A394601F090
:1027C0003FFC002800F0ED8032463B46304639465B
:1027D00001F086F97CA3D3E9002304460D4601F0FD
:1027E0007FF97BA3D3E9002300F0C4FF22462B46E8
:1027F00001F076F978A3D3E9002300F0B9FF22466F
:102800002B4601F06DF976A3D3E9002300F0B2FF67
:1028100022462B4601F064F973A3D3E9002300F0AC
:10282000A7FF22462B4601F05BF971A3D3E90023F1
:1028300000F0A0FF22462B4601F052F982468B465B
:102840000022714B2046294601F04AF95246804643
:1028500089465B462046294601F042F953EC182B85
:1028600004460D463046394601F03AF902460B4619
:102870002046294600F07CFF02460B46404649466A
:1028800000F076FF02460B460020604900F070FF22
:1028900041EC100B03B0BDEC028BBDE8F08F10EEE5
:1028A000102A10EE100A3B46394601F019F946A3EA
:1028B000D3E9002304460D4601F012F944A3D3E9FD
:1028C000002300F057FF22462B4601F009F942A3EE
:1028D000D3E9002300F04CFF22462B4601F000F91B
:1028E0003FA3D3E9002300F045FF22462B4601F029
:1028F000F7F83DA3D3E9002300F03AFF22462B4628
:1029000001F0EEF83AA3D3E9002300F033FF2B46A1
:10291000224601F0E5F83E4B994582468B468FDD15
:102920003C4B994544DC0022A9F5001300203749AF
:102930009046994600F01CFFCDE900010022324B81
:102940002046294601F0CCF842464B4600F010FFE5
:102950005246804689465B462046294601F0C0F82B
:1029600053EC182B04460D463046394601F0B8F8B2
:1029700002460B462046294600F0FAFE02460B4668
:102980004046494600F0F4FE02460B46DDE90001F0
:1029900000F0EEFE41EC100B03B0BDEC028BBDE885
:1029A000F08F9FED150B03B0BDEC028BBDE8F08FEF
:1029B0009FED137B4FF000088DED007BDFF8589002
:1029C000BCE700BFAFF30080D43888BEE9FAA8BDE9
:1029D000C4B1B4BD9EEE213EAD529C804F7E923E6E
:1029E0009015CB19A001FA3E7751C1166CC1563F24
:1029F0004C5555555555A53F000000000000F03FCF
:102A0000000000000000E73F0000E03F0000F03F52
:102A10003233D33F0000E93F0000D23F0000000006
:102A20002DE9F04FADF5197DC14CA29EC14D54F872
:102A300026600793D41E85FB0475E417C4EBA50438
:102A400024EAE4741D46631CA3EB8303013D02EBFF
:102A5000C3030593731904960994019503900B9190
:102A6000A4EB05071AD43B44002400255E1C0DF19D
:102A70008008DDF88C9208E059F8270000F0C6FFC6
:102A80000137B742E8E8020108D0002FF4DA013735
:102A900020462946B742E8E80201F6D1049B002B04
:102AA000079B4FEAC30302932ADB039A20A902EB98
:102AB000030801EB0309049B72AA02EBC30B0DF59B
:102AC000E07A019B002B4FF000064FF0000711DB6E
:102AD000039C4D4675E90223F4E8020101F000F879
:102AE00002460B463046394600F044FE4445064651
:102AF0000F46EFD1EAE80267DA4509F10809E0D1AB
:102B0000DDE90204049920448B0082460BA8A3F15E
:102B10000802C31808930CAB13440A938B4698AB76
:102B200003EBCB03BBF1000F53E9284529DD70AB64
:102B300003EBCB080DF1300900227F4B20462946DC
:102B400000F0CEFF01F07CFA00F060FF00227B4B2A
:102B500006460F4600F0C4FF02460B4620462946B3
:102B600000F006FE01F06CFA78E9022349F8040B44
:102B70003946304600F0FEFD70AB984504460D46E0
:102B8000DAD1DDF8149045EC104B484600F04CFDCE
:102B900055EC104B00224FF07F5310EE100A2946DF
:102BA00000F09EFF41EC100B00F022FC002251ECE3
:102BB000100B634B00F094FF02460B46204629465B
:102BC00000F0D6FD0D46044601F03AFA804600F0CA
:102BD0001DFF0B4602462946204600F0C9FD4B4624
:102BE000002B06460F4640F3E0800BF1FF320CA9A4
:102BF000C9F1180351F8225045FA03F101FA03F321
:102C00000CA8EB1A40F82230C9F11705884443FAA2
:102C100005F5002D2CDDBBF1000F08F1010840F394
:102C200086820C9C002C40F0A680BBF1010F0AD0DC
:102C30000CA9012251F8044F531C002C40F09D8038
:102C40009B451A46F6D1059B002B0EDD012B00F0AB
:102C5000D880022B09D10BF1FF320CAB0CA953F831
:102C60002230C3F3150341F82230022D00F0AE806C
:102C7000002200233046394601F09AF9002800F07E
:102C80005882049B0BF1FF394B4510DC0BF180435C
:102C90000CAA013B089802EB8303002253F80419A5
:102CA000834242EA0102F9D1002A40F0B580049B38
:102CB0000CAA013B52F82330002B40F0A0800A9A66
:102CC000012352F8041901330029FAD05B440BF1B7
:102CD0000109994506934BDC099A079909EB02080B
:102CE00001EB0B0508F1804802EB030BA39B08F1F5
:102CF000FF3803EB880870AB03EBC909A39B20A93D
:102D000003EB8B0301EBC505029358F8040F00F0A9
:102D10007DFE0B4601990246002905F1080BC5E925
:102D200000234FF000064FF000071BDB039C0BE075
:102D300048B00008ABAAAA2A0000703E000070410B
:102D40000000204075E90223F4E8020100F0C8FE0B
:102D500002460B463046394600F00CFD5445064607
:102D60000F46EFD1029B9845E9E802675D46CCD15A
:102D7000DDF818B0D3E6012300220CA9C4F1807459
:102D80009B4541F822400EDD51F8232001EB8B00DA
:102D900001EB83036FF07F4100E01A688A1A43F861
:102DA000042B8342F9D101244DE706D10BF1FF3307
:102DB0000CAA52F82350ED152BE700227E4B01F0B0
:102DC00015F9002840F0A981054651E732463B46F7
:102DD00000207A4900F0CCFC06460F46002C3FF458
:102DE00047AF05989FED700B00F01EFC304639464A
:102DF00053EC102B00F0BCFC06460F4638E70123CD
:102E000064E70BF1FF320CAB0CA953F82230C3F38B
:102E1000160341F8223028E70CAB059A53F8293005
:102E2000183ACDE9068505926BB909F18043013B5B
:102E30000CA901EB830353F8041909F1FF39183A7F
:102E40000029F8D0059205989FED570B00F0ECFB98
:102E5000B9F1000F55EC104BC0F2C9814FEAC9031C
:102E600070AA02EB030808930CAB03EB8906DFF8AA
:102E700050B14FF0000A08F10807043656F8040D67
:102E800000F0C4FD22462B4600F02AFE5B4667E9AF
:102E9000020152462046294600F022FE0CAB9E421B
:102EA00004460D46EAD148AB03930193CDF8149044
:102EB00009F10103DDF810900293C3464FF0000AB8
:102EC000B9F1000FC0F23081DFF8F8805D4638A319
:102ED000D3E9002300260027002403E0544510DC3A
:102EE000F8E80223F5E8020100F0FAFD02460B467D
:102EF0003046394600F03EFC0134A14506460F46F7
:102F0000ECDA019BE3E802670193029B0AF1010AF4
:102F10009A45ABF1080BD3D1A29BDDF81490032B9B
:102F200039D8DFE813F0DF0006000600530048AB95
:102F30000393B9F1000F4FF000004FF0000109DBDF
:102F4000039D05EBC904083474E9022300F012FC68
:102F5000A542F9D1079B002B40F027810B9BC3E9C9
:102F600000010B4603990246D1E9000100F000FC84
:102F7000B9F1000F0CDD4AAD01240134F5E802235C
:102F800000F0F8FBA145F8DA079B002B40F01D810B
:102F90000B9BC3E90201069B03F007000DF5197DA9
:102FA000BDE8F08FAFF30080000000000000F03FAC
:102FB00000000040FB21F93F0000E03F0000F03F2F
:102FC0000000703E60B0000848AB0393B9F1000FF9
:102FD00040F32981039ACDF810904FEAC903019379
:102FE000D318D3E900AB09F10053013B02EBC90848
:102FF0000293914678E9026752465B46304639466D
:1030000000F0B8FB04460D4602460B4630463946F2
:1030100000F0AEFB52465B4600F0ACFBC145A24659
:10302000AB46C8E90201C8E90045E3D1DDF81090DC
:10303000B9F1010F40F3F780019B039A0299134401
:10304000C900D3E9006701F1080A019192440DF526
:10305000947B7AE9028932463B464046494600F075
:1030600089FB04460D4602460B464046494600F0A1
:103070007FFB32463B4600F07DFBD34526462F467C
:10308000CAE90201CAE90045E3D1019C039B10345F
:10309000002000211C4403F1100574E9022300F014
:1030A00069FBA542F9D1039C079ED4E90023D4E92A
:1030B0000245002E00F08D8003F1004701F100432E
:1030C0000B99C1E90403069B2646944605F100448A
:1030D00003F00700C1E900C7C1E902640DF5197DDD
:1030E000BDE8F08F089C039D0834002000212C448B
:1030F00074E9022300F03EFBA542F9D1079B13B10E
:1031000001F1004319460B9BC3E90001069B03F044
:1031100007000DF5197DBDE8F08FBBF1000F08F138
:10312000010876DD02257CE500260027E9E600247B
:1031300089E5CDE90685059D47EC106B684200F0F6
:1031400073FA57EC106B0022384B10EE100A394618
:1031500000F04CFF00B30022354B3046394600F0FA
:10316000BFFC00F06DFF044600F050FC00222F4B26
:1031700000F0B6FC0B4602463946304600F0F8FA3D
:1031800000F05EFF0BF101090CAB183543F82B0082
:10319000059543F8294056E63046394600F050FF81
:1031A0000CABD94643F82B004DE60B9C01F10043D4
:1031B000C4E900030B4603990246D1E9000100F07F
:1031C000D7FAB9F1000F3FF7D6AE01F10043194627
:1031D000DEE60B9EC6E90023069BC6E9040103F068
:1031E0000700C6E902450DF5197DBDE8F08FA29BE9
:1031F000032B3FF6D0AE01A252F823F00D320008A7
:103200002F2F00082F2F0008C92F000800200021B1
:1032100074E732463B460020064900F0A9FA022531
:1032200006460F4624E5002000213CE700007041DF
:103230000000703E0000F03F2DE9F04F55EC104BC0
:103240002DED028BB0EE418AF0EE618A25F000434D
:10325000B3F1795F83B0824607DA10EE100A29468F
:1032600000F0EEFE002800F08E8022462B4620461D
:10327000294600F035FC06460F4602460B4620461E
:10328000294600F02DFC47A3D3E900238046894658
:103290003046394600F024FC44A3D3E9002300F073
:1032A00067FA32463B4600F01BFC42A3D3E90023F9
:1032B00000F060FA32463B4600F012FC3FA3D3E92F
:1032C000002300F055FA32463B4600F009FC3DA3CE
:1032D000D3E9002300F04EFACDE90001BAF1000F66
:1032E00037D000222E4B51EC180B00F0F9FBDDE932
:1032F000002382468B464046494600F0F1FB0246D9
:103300000B465046594600F033FA32463B4600F031
:10331000E7FB53EC182B00F02BFA1FA3D3E9002393
:1033200006460F464046494600F0DAFB02460B4689
:103330003046394600F01EFA02460B462046294622
:1033400000F016FA41EC100B03B0BDEC028BBDE8A7
:10335000F08F02460B463046394600F0C1FB0EA303
:10336000D3E9002300F004FA42464B4600F0B8FBD4
:1033700022462B4600F0FEF941EC100B03B0BDECE9
:10338000028BBDE8F08F45EC104B03B0BDEC028B17
:10339000BDE8F08FAFF30080495555555555C53FF1
:1033A0000000E03F7CD5CF5A3AD9E53DEB9C2B8A13
:1033B000E6E55A3E7DFEB157E31DC73ED561C11912
:1033C000A0012A3FA6F810111111813F51EC100BFA
:1033D00010EE102A21F0004343EC102B704700BF81
:1033E00010EE903A43F0004000F58010C00F704797
:1033F00051EC100BC1F30A532DE9F041A3F2FF3554
:10340000132D0C460F4610EE106A1DDC002D3DDB1F
:10341000394B43FA05F801EA0803034319D034A3F2
:10342000D3E9002300F0A6F90022002300F0E8FD14
:10343000D0B3002C04DA4FF4801343FA05F52F447F
:1034400027EA080400262FE0332D06DDB5F5806F4E
:1034500030D041EC100BBDE8F081A3F213434FF0E4
:10346000FF3828FA03F818EA000FF2D020A3D3E9B6
:10347000002300F07FF90022002300F0C1FD98B185
:10348000002C28DB26EA08063C460DE018A3D3E909
:10349000002300F06FF90022002300F0B1FD18B105
:1034A000002C0FDB002634462346324643EC102B1B
:1034B000BDE8F08110EE102A0B4600F05BF941ECFC
:1034C000100BC8E724F000430C4A1E43002E18BF1F
:1034D00014460026E8E7142D08D00123C5F1340571
:1034E00003FA05F5AE1928BFFF18CBE70137C9E786
:1034F0009C7500883CE4377EFFFF0F000000F0BFA2
:1035000000207047000000009FED010B704700BFD6
:10351000000000000000F87FF0B551EC100BC1F383
:103520000A55A5F2FF32132A83B00B464FEAD17633
:1035300010EE104A2FDC002A4ADB394D154101EA12
:103540000507074323D06D0829400C430CD04FF4E6
:103550008021132A23EA050541FA02F343EA050311
:103560000CBF4FF0004400242E4A02EBC606204652
:10357000D6E9004502462946204600F0FBF8CDE991
:10358000000122462B46DDE9000100F0F1F841EC94
:10359000100B03B0F0BD332A07DDB2F5806FF6D112
:1035A00010EE102A00F0E6F8F1E7A5F213454FF00F
:1035B000FF32EA401042EAD052081042D4D04FF015
:1035C000804124EA020241FA05F542EA0504CBE70C
:1035D00021F000420243DAD0C1F313020243544205
:1035E000104D1443240B05EBC6004F0C04F40021CE
:1035F000D0E900457F0410EE102A41EA0703204677
:10360000294600F0B7F8CDE900012B462246DDE956
:10361000000100F0ADF821F0004343EAC671B6E7BF
:10362000FFFF0F0098B0000838B553EC102BC3F320
:103630000A511C46054629BB10EE101A23F000441F
:1036400021431ED0194600223D4B3E4C10EE100A7D
:1036500000F046FAA54202460B463BDB0C46C1F39E
:103660000A513639294440F2FE70814216DC0029A5
:1036700021DD24F0FF4424F4E00444EA015343EC48
:10368000102B38BD40F2FF708142EBD110EE100AD2
:10369000194600F06FF841EC100B38BD002B20A14B
:1036A000D1E900011EDB1EA3D3E9002300F018FAC4
:1036B00041EC100B38BD11F1350F1EDA4CF25031D0
:1036C0008D42EBDC002B18A1D1E9000102DA18A130
:1036D000D1E9000114A3D3E9002300F001FA41EC81
:1036E000100B38BD14A1D1E900010DA3D3E90023CB
:1036F00000F0F6F941EC100BDCE724F0FF4424F471
:10370000E004363144EA01531046194600220E4BBC
:1037100000F0E6F941EC100B38BD00BFAFF30080BC
:103720009C7500883CE4377E59F3F8C21F6EA501F2
:1037300059F3F8C21F6EA5819C7500883CE437FEE2
:1037400000005043B03CFFFF0000903C044A054994
:103750001368002B08BF0B461844106018467047CA
:10376000980600204874002081F0004102E000BF6C
:1037700083F0004330B54FEA41044FEA430594EA31
:10378000050F08BF90EA020F1FBF54EA000C55EA6C
:10379000020C7FEA645C7FEA655C00F0E2804FEA3D
:1037A0005454D4EB5555B8BF6D420CDD2C4480EA1F
:1037B000020281EA030382EA000083EA010180EA4F
:1037C000020281EA0303362D88BF30BD11F0004F9D
:1037D0004FEA01314FF4801C4CEA113102D04042D3
:1037E00061EB410113F0004F4FEA03334CEA13330E
:1037F00002D0524263EB430394EA050F00F0A78026
:10380000A4F10104D5F1200E0DDB02FA0EFC22FA20
:1038100005F2801841F1000103FA0EF2801843FA14
:1038200005F359410EE0A5F120050EF1200E012A05
:1038300003FA0EFC28BF4CF0020C43FA05F3C01843
:1038400051EBE37101F0004507D54FF0000EDCF1BC
:10385000000C7EEB00006EEB0101B1F5801F1BD365
:10386000B1F5001F0CD349085FEA30004FEA3C0C69
:1038700004F101044FEA445212F5800F80F09A805F
:10388000BCF1004F08BF5FEA500C50F1000041EB63
:10389000045141EA050130BD5FEA4C0C404141EB67
:1038A000010111F4801FA4F10104E9D191F0000F8E
:1038B00004BF01460020B1FA81F308BF2033A3F111
:1038C0000B03B3F120020CDA0C3208DD02F1140C08
:1038D000C2F10C0201FA0CF021FA02F10CE002F143
:1038E0001402D8BFC2F1200C01FA02F120FA0CFC3C
:1038F000DCBF41EA0C019040E41AA2BF01EB045185
:10390000294330BD6FEA04041F3C1CDA0C340EDC82
:1039100004F11404C4F1200220FA04F001FA02F3C5
:1039200040EA030021FA04F345EA030130BDC4F183
:103930000C04C4F1200220FA02F001FA04F340EA78
:103940000300294630BD21FA04F0294630BD94F029
:10395000000F83F4801306BF81F480110134013D10
:103960004EE77FEA645C18BF7FEA655C29D094EA81
:10397000050F08BF90EA020F05D054EA000C04BFFF
:103980001946104630BD91EA030F1EBF00210020EA
:1039900030BD5FEA545C05D14000494128BF41F089
:1039A000004130BD14F580043CBF01F5801130BDED
:1039B00001F0004545F0FE4141F470014FF0000078
:1039C00030BD7FEA645C1ABF194610467FEA655C29
:1039D0001CBF0B46024650EA013406BF52EA0335CB
:1039E00091EA030F41F4002130BD00BF90F0000FB9
:1039F00004BF0021704730B54FF4806404F13204F5
:103A00004FF000054FF0000150E700BF90F0000FAD
:103A100004BF0021704730B54FF4806404F13204D4
:103A200010F0004548BF40424FF000013EE700BFA4
:103A300042004FEAE2014FEA31014FEA02701FBF34
:103A400012F07F4393F07F4F81F06051704732F066
:103A50007F4208BF704793F07F4F04BF41F40021BD
:103A6000704730B54FF4607401F0004521F000411B
:103A70001CE700BF50EA010208BF704730B54FF0A5
:103A800000050AE050EA010208BF704730B511F0A6
:103A9000004502D5404261EB41014FF4806404F1DE
:103AA00032045FEA915C3FF4D8AE4FF003025FEA64
:103AB000DC0C18BF03325FEADC0C18BF033202EBE8
:103AC000DC02C2F1200300FA03FC20FA02F001FA42
:103AD00003FE40EA0E0021FA02F11444BDE600BFE5
:103AE00070B54FF0FF0C4CF4E06C1CEA11541DBF94
:103AF0001CEA135594EA0C0F95EA0C0F00F0DEF85F
:103B00002C4481EA030621EA4C5123EA4C5350EA43
:103B1000013518BF52EA033541F4801143F4801394
:103B200038D0A0FB02CE4FF00005E1FB02E506F025
:103B30000042E0FB03E54FF00006E1FB03569CF07A
:103B4000000F18BF4EF0010EA4F1FF04B6F5007F80
:103B500064F5407404D25FEA4E0E6D4146EB0606F2
:103B600042EAC62141EA55514FEAC52040EA5E507B
:103B70004FEACE2EB4F1FD0C88BFBCF5E06F1ED825
:103B8000BEF1004F08BF5FEA500E50F1000041EB5C
:103B9000045170BD06F0004646EA010140EA020009
:103BA00081EA0301B4EB5C04C2BFD4EB0C0541EA2B
:103BB000045170BD41F480114FF0000E013C00F340
:103BC000AB8014F1360FDEBF002001F0004170BD64
:103BD000C4F10004203C35DA0C341BDC04F114047D
:103BE000C4F1200500FA05F320FA04F001FA05F209
:103BF00040EA020001F0004221F0004110EBD370D6
:103C000021FA04F642EB06015EEA430E08BF20EA01
:103C1000D37070BDC4F10C04C4F1200500FA04F3A4
:103C200020FA05F001FA04F240EA020001F0004136
:103C300010EBD37041F100015EEA430E08BF20EAA9
:103C4000D37070BDC4F1200500FA05F24EEA020EF1
:103C500020FA04F301FA05F243EA020321FA04F020
:103C600001F0004121FA04F220EA020000EBD370D7
:103C70005EEA430E08BF20EAD37070BD94F0000FD7
:103C80000FD101F00046400041EB010111F4801F0B
:103C900008BF013CF7D041EA060195F0000F18BFBC
:103CA000704703F00046520043EB030313F4801FF8
:103CB00008BF013DF7D043EA0603704794EA0C0FB2
:103CC0000CEA135518BF95EA0C0F0CD050EA4106C8
:103CD00018BF52EA4306D1D181EA030101F0004145
:103CE0004FF0000070BD50EA410606BF104619466D
:103CF00052EA430619D094EA0C0F02D150EA013679
:103D000013D195EA0C0F05D152EA03361CBF1046B9
:103D100019460AD181EA030101F0004141F0FE4158
:103D200041F470014FF0000070BD41F0FE4141F4DC
:103D3000780170BD70B54FF0FF0C4CF4E06C1CEADC
:103D400011541DBF1CEA135594EA0C0F95EA0C0F91
:103D500000F0A7F8A4EB050481EA030E52EA03354C
:103D60004FEA013100F088804FEA03334FF080556D
:103D700045EA131343EA12634FEA022245EA11159A
:103D800045EA10654FEA00260EF000419D4208BF4B
:103D9000964244F1FD0404F5407402D25B084FEAF8
:103DA0003202B61A65EB03055B084FEA32024FF4A4
:103DB00080104FF4002CB6EB020E75EB030E22BF01
:103DC000B61A754640EA0C005B084FEA3202B6EBC1
:103DD000020E75EB030E22BFB61A754640EA5C0070
:103DE0005B084FEA3202B6EB020E75EB030E22BF00
:103DF000B61A754640EA9C005B084FEA3202B6EB01
:103E0000020E75EB030E22BFB61A754640EADC00BF
:103E100055EA060E18D04FEA051545EA16754FEA21
:103E200006164FEAC30343EA52734FEAC2025FEA3F
:103E30001C1CC0D111F4801F0BD141EA00014FF0CE
:103E400000004FF0004CB6E711F4801F04BF01439F
:103E50000020B4F1FD0C88BFBCF5E06F3FF6AFAEBB
:103E6000B5EB030C04BFB6EB020C5FEA500C50F14B
:103E7000000041EB045170BD0EF0004E4EEA1131CE
:103E800014EB5C04C2BFD4EB0C0541EA045170BDD5
:103E900041F480114FF0000E013C90E645EA060E19
:103EA0008DE60CEA135594EA0C0F08BF95EA0C0F47
:103EB0003FF43BAF94EA0C0F0AD150EA01347FF48F
:103EC00034AF95EA0C0F7FF425AF104619462CE766
:103ED00095EA0C0F06D152EA03353FF4FDAE1046C9
:103EE000194622E750EA410618BF52EA43067FF41A
:103EF000C5AE50EA41047FF40DAF52EA43057FF4AA
:103F0000EBAE12E74FF0FF3C06E000BF4FF0010CB4
:103F100002E000BF4FF0010C4DF804CD4FEA410C18
:103F20007FEA6C5C4FEA430C18BF7FEA6C5C1BD0E5
:103F300001B050EA410C0CBF52EA430C91EA030F66
:103F400002BF90EA020F0020704710F1000F91EAC3
:103F5000030F58BF994208BF90422CBFD8176FEA91
:103F6000E37040F0010070474FEA410C7FEA6C5C5F
:103F700002D150EA013C07D14FEA430C7FEA6C5C66
:103F8000D6D152EA033CD3D05DF8040B704700BF92
:103F90008446104662468C461946634600E000BFE0
:103FA00001B5FFF7B7FF002848BF10F1000F01BDB2
:103FB0004DF808EDFFF7F4FF0CBF012000205DF87D
:103FC00008FB00BF4DF808EDFFF7EAFF34BF012002
:103FD00000205DF808FB00BF4DF808EDFFF7E0FF9B
:103FE00094BF012000205DF808FB00BF4DF808EDEC
:103FF000FFF7CEFF94BF012000205DF808FB00BF53
:104000004DF808EDFFF7C4FF34BF012000205DF834
:1040100008FB00BF4FEA410C7FEA6C5C02D150EA1A
:10402000013C0AD14FEA430C7FEA6C5C02D152EAB0
:10403000033C02D14FF0000070474FF00100704781
:104040004FEA410212F5001215D211D56FF47873C0
:10405000B3EB625212D94FEAC12343F0004343EA63
:10406000505311F0004F23FA02F018BF404270473E
:104070004FF00000704750EA013005D111F00040C8
:1040800008BF6FF0004070474FF00000704700BF5E
:104090007BB972B90029BEBF00204FF0004106E095
:1040A00008BF00281CBF6FF000414FF0FF3000F048
:1040B000BDB9ADF1080C6DE904CE002909DB002B78
:1040C0001ADB00F04DF8DDF804E0DDE9022304B06E
:1040D0007047404261EB4101002B1BDB00F040F8D0
:1040E000DDF804E0DDE9022304B0404261EB410168
:1040F000524263EB43037047524263EB430300F0C9
:104100002FF8DDF804E0DDE9022304B0404261EB62
:1041100041017047524263EB430300F021F8DDF8A0
:1041200004E0DDE9022304B0524263EB430370472D
:1041300053B94AB9002908BF00281CBF4FF0FF310E
:104140004FF0FF3000F072B9ADF1080C6DE904CE0C
:1041500000F006F8DDF804E0DDE9022304B0704762
:104160002DE9F047089E04468846002B4BD18A4231
:10417000154667D9B2FA82F24AB1C2F1200701FAB4
:1041800002F320FA07F7954047EA030894404FEA04
:10419000154E230CB8FBFEF71FFA85FC0EFB1788A3
:1041A00043EA084307FB0CF1994209D9EB1807F1E0
:1041B000FF3080F01B81994240F21881023F2B446E
:1041C0005B1AA4B2B3FBFEF00EFB103344EA0344C7
:1041D00000FB0CFCA44509D92C1900F1FF3380F039
:1041E0000781A44540F2048102382C4440EA07408C
:1041F000A4EB0C0400271EB1D4400023C6E9004301
:104200003946BDE8F0878B4209D9002E00F0EB80DB
:104210000027C6E9000138463946BDE8F087B3FA01
:1042200083F7002F47D18B4202D3824200F2FA80FB
:10423000841A61EB030301209846002EE0D0C6E902
:104240000048DDE702B9FFDEB2FA82F2002A40F050
:104250008F80491B4FEA154E1FFA85F80127B1FBE5
:10426000FEFC230C0EFB1C1143EA014308FB0CF17E
:10427000994207D9EB180CF1FF3002D2994200F2B3
:10428000CD808446591AA3B2B1FBFEF00EFB101488
:1042900043EA044408FB00F8A04507D92C1900F1B3
:1042A000FF3302D2A04500F2B6801846A4EB080402
:1042B00040EA0C409FE7C7F1200CBB4022FA0CFEFD
:1042C0004EEA030E01FA07F420FA0CF521FA0CF37A
:1042D0004FEA1E482543B3FBF8F92C0C08FB1933B1
:1042E0001FFA8EFA44EA034309FB0AF49C4202FADD
:1042F00007F200FA07F10BD91EEB030309F1FF30B7
:1043000080F087809C4240F28480A9F102097344C6
:104310001B1BADB2B3FBF8F008FB103345EA0344B6
:1043200000FB0AFAA24508D91EEB040400F1FF3392
:104330006BD2A24569D90238744440EA0940A0FB17
:104340000289A4EB0A044C45C2464B4654D351D0D3
:10435000002E69D0B1EB0A0564EB030404FA0CFCEF
:10436000FD40FC404CEA0505C6E90054002747E73C
:10437000C2F1200320FA03F7954001FA02F021FA76
:1043800003F34FEA154E3843010CB3FBFEF71FFA57
:1043900085F80EFB173341EA034107FB08F38B4214
:1043A00004FA02F407D9691807F1FF3C2FD28B42B7
:1043B0002DD9023F2944CB1A81B2B3FBFEF00EFB8C
:1043C000103341EA034100FB08F38B4207D9691817
:1043D00000F1FF3C17D28B4215D902382944C91A83
:1043E00040EA07473BE73746304609E70746E7E636
:1043F0001846FBE64145ABD2B8EB020A69EB0E0268
:1044000001381346A4E76046E9E7184695E7674692
:10441000D1E781467CE702382C4447E7ACF1020C37
:104420002B442FE7384608E73746E9E6704700BFD8
:10443000014B1868704700BF000000200368B3F10B
:10444000A04F02D1014B01221A707047480D002085
:104450000368B3F1A04F02D1014B01221A607047EB
:10446000E81200200349044B0020012208701A7052
:10447000704700BFD81200206C0C00200249034A8C
:1044800001230B7013707047D81200206C0C0020B1
:1044900008B52021044804F0E3FB0449044B002044
:1044A000012208701A7008BD00040048003C00207A
:1044B000013C002008B52021044804F0D1FB044948
:1044C000044A01230B70137008BD00BF00040048AC
:1044D000003C0020013C00200268034B9A4202D1BC
:1044E000024B01221A70704700140040F80C0020A3
:1044F00038B5084B984200D038BD074D044628789F
:1045000000F02AFC294620460122BDE8384005F08B
:1045100019BC00BFDC0B0020FC1B002010B50B4BAE
:104520000B4C0C4882B001221A7005F05FF920464E
:10453000102104F0A5FE0023009320464FF40063F1
:10454000054A102104F0E2FE02B010BDF81A002066
:10455000600A0020140A0020001C002010B5084B3F
:10456000084C094800221A7005F074F92046102101
:1045700004F0BAFE20461021BDE8104004F048BF08
:10458000F81A0020600A0020140A002030B50D4BF4
:104590000D490E4C0E4883B04FF4806201251D700A
:1045A00002F076FD0B4805F021F92046002104F0C9
:1045B00067FE0021204600918023074A04F0A6FEF2
:1045C00003B030BDFE1B0020F0120020600A002066
:1045D000700B0020FC0C0020D410002038B50A4BD2
:1045E0000A4D0B4800241C7003F066FB094805F0D7
:1045F00031F92146284604F077FE21462846BDE8D9
:10460000384004F005BF00BFFE1B0020600A0020F8
:10461000700B0020FC0C002008B5184806F0FCFBCD
:10462000174B1B68023B042B04D8DFE803F0131878
:104630001D0E2200114B00229A62104806F04EFB1C
:104640000E48BDE8084006F0CDBB0C4B4FF480325D
:104650009A62F2E7094B4FF480429A62EDE7074B0A
:104660004FF400429A62E8E7044B4FF440429A62EA
:10467000E3E7024B4FF4A0329A62DEE7D40A00204F
:10468000F41A002030B50021A5B00C46382205A848
:10469000FBF7C8FE2146442213A8CDE90044CDE92A
:1046A00002440494FBF7BEFE204604F09FFC032462
:1046B000022301254FF480311C2205A8CDE90551C4
:1046C0000C930E93CDE9103312930D940F9203F0D7
:1046D00077FC08B172B6FEE703460F226846042154
:1046E000CDE90143CDE90333009203F0BBFE03465D
:1046F00008B172B6FEE748F201014FF0005213A86C
:10470000CDE91313229204F07DF808B172B6FEE7EA
:1047100025B030BD2DE98048DFF8ECA2AE4DAF4F9B
:104720009FB00024AAF8004001F046FA00F0CCFB4C
:1047300001F094F901F0BEF901F0E6F903F008FC8C
:10474000FFF7A0FFCDE91244CDE914441694EB6CB9
:10475000A34843F02003EB64EB6C03F020030593C4
:10476000059BEB6C43F00103EB64EB6C03F001037E
:104770000693069BEB6C43F00203EB64EB6C03F0D7
:104780000203224620210793079B8846012604F056
:1047900061FA12A99248CDE91444CDE9128604F0D9
:1047A0007DF9AB6C43F00403AB64AB6C03F0040322
:1047B0000393039BAB6C3343AB64AB6C3340224637
:1047C000214604930B20049B04F0A8FC0B2004F06A
:1047D000DBFC224621460C2004F0A0FC0C2004F057
:1047E000D3FC224621460E2004F098FC0E2004F053
:1047F000CBFC224621460F2004F090FC0F2004F051
:10480000C3FC214612A83022FBF70CFE754B3B601F
:10481000384604F01FFD08B172B6FEE700241E25DD
:10482000CDE91445002400250223CDE916450246B2
:104830008DF84C0012A901240025384612938DF8FA
:104840004D60CDE9184504F02FFE034608B172B65D
:10485000FEE73846102212A98DF84D30159304F06A
:1048600023FE054608B172B6FEE75F4C089001468C
:10487000424612A80B95CDE90955CDE90C55CDE975
:104880000E55CDE910550427FBF7CCFD4FF440330E
:104890004FF0A0422046C4E90023C4E90255C4E910
:1048A000045525776677266284F82450C4E90B55B1
:1048B00084F83860E56384F84060C4E91155E56424
:1048C0002665A76102F0D4FA034608B172B6FEE786
:1048D00008A92046089303F0A7FA08B172B6FEE7CC
:1048E000424B0B9340F6F9714FF4400305220C93B1
:1048F0000F914FF480533E4D11930BA920460D9517
:10490000109203F013F8034608B172B6FEE7204692
:104910007F22062412A912951497169717931394C1
:10492000159202F0CDFD08B172B6FEE7314C324966
:10493000129040F2E73340F28F62CDE91300A0609D
:10494000A0612046E3602160626004F0B1FE03468E
:1049500008B172B6FEE7204612A91293149305F02F
:104960008FF908B172B6FEE7244B25491490CDE9C2
:104970001200C3E90100986141F6FF521846196020
:10498000DA6004F095FE08B172B6FEE700234FF03E
:10499000200812A919481493CDF8488005F070F941
:1049A000034608B172B6FEE7DFF86090154A13902F
:1049B0001493CDE9163348464FF4001301264027DF
:1049C000C9F8002012961897159304F005FC0546C7
:1049D000F0B172B6FEE700BF00100240600A00208E
:1049E0000004004800080050700B00200000C07D4B
:1049F000002090B64C0D002000140040FC0C00205C
:104A000000100040000C0240F01A0020D00C0020E2
:104A1000A04C12A9484604F0F9FB9F4921604FF4CD
:104A2000E1320C232046A560C4E90355C4E90655CC
:104A3000C4E90855A5626260636105F097FE01460E
:104A400008B172B6FEE7204606F0CCF8014608B180
:104A500072B6FEE7204606F003F908B172B6FEE72B
:104A6000204606F0A1F808B172B6FEE78B4C8C4ADE
:104A70000D90CDE91200CDE91400CDE90B00C4E999
:104A80000100C4E90400A061EF2320462260E36036
:104A900004F00EFE08B172B6FEE74FF4805312A97F
:104AA0002046129304F024FF034608B172B6FEE7D5
:104AB0000BA92046CDE90B830D9305F0E1F808B171
:104AC00072B6FEE7774B784D186180244FF40031C1
:104AD0009861D8624FF4A03218469F601E751D6021
:104AE0005C60C3E9091206F0F9F808B172B6FEE796
:104AF00000F00EFD00F052FD6A48DFF81492DFF876
:104B000014826A4FDFF810B2694D6A4E6A4C06F0A3
:104B100069F9FFF781FD694804F0B0FE0122684998
:104B20005C4805F00FF9FFF731FD99F80030002BD4
:104B300039D098F80030ABB101222021614804F04F
:104B400089F83B680093604A604B61484FF480618C
:104B500000F072FA002220215A4804F07BF800236A
:104B600088F800305B4B1B78EBB15B4B1B68002B6C
:104B700000F089805A1E012A40F2D080032B05D113
:104B8000234640225149504800F03AFC534B5449C7
:104B90001A78544801EB02224023214602F006F91C
:104BA0004C4A00231370504B1B781BB34F4B1B78A0
:104BB0007BB14F4B444A18783B6800934D4B4FF400
:104BC000806103EB0030414B00F0BAF9474A002303
:104BD0001370494B1B786BB13F4B1B683BB35A1E9C
:104BE000012A1BD9032B05D12346402237493648D9
:104BF00000F00CFA414B1B78002B96D099F800304E
:104C00001BB14021304800F02BFD3D4B1A783D4B45
:104C10001B789A4211D000F0AFF8F6E73A4B0093B8
:104C2000402223462949284800F0ACF9E2E7224611
:104C30004021254800F0D2F9DCE7BAF800300BB18A
:104C400000F062FFBBF8002032B13049114805F096
:104C50002DF90023ABF8003032682B6852B10BB944
:104C600001F094F80022312332602B60234A0023A4
:104C700013705AE7002BF9D0013B2B60002BF5D1C4
:104C800001F084F8F2E7224640210F4800F028FCAA
:104C90007CE700BFDC0B002000380140140A002034
:104CA00000340140D40A002000030140E01200203B
:104CB000CC100020E8120020FC1A00204C0D00202F
:104CC000FC1B002000040048043C0020CC0F002006
:104CD000F01200206C0C0020B80F0020D812002029
:104CE000D41000201C690020F81A0020013C00208C
:104CF000003C0020001C0020144F0020F80C002075
:104D0000E5120020E412002047E17A14B80D0020DB
:104D1000FE1B0020480D0020BC0F0020044B009318
:104D2000402223460349044800F086FB2EE700BFDB
:104D300047E17A14CC0F0020043C002072B6FEE755
:104D400003780133194001700846704780FB010168
:104D500001F31E004000704710B4054A054C11785D
:104D60004B1C03F01F03137060545DF8044B704735
:104D7000E5120020980D002010B5064C064A237855
:104D8000D05C00F05FFD2378013303F01F03237034
:104D900010BD00BFE4120020980D0020E1B1F0B476
:104DA0000E4E0F4F32880378BB54013292B2B2F5E7
:104DB000007F32800ED0002306E0C55CBD54A2B255
:104DC000B2F5007F328005D00133DBB28B4202F1B5
:104DD0000104F2D3F0BC7047704700BFBC0F002045
:104DE000B80D002008B50A4B0A4A1B681168022B4F
:104DF0000BD0012B08BFA1F21E710023064A002030
:104E0000FFF746F9054B186008BD01F21E71F4E783
:104E1000B80F0020C00F002030570500E01200201E
:104E2000044B054A05491B7812680968044800F0DC
:104E3000CBBB00BFEC120020043D0020C40F0020BB
:104E40003C72002008B500F063FB0A4B0A4A1B685D
:104E50001168022B0BD0012B08BFA1F21E71002399
:104E6000064A0020FFF714F9054B186008BD01F24F
:104E70001E71F4E7B80F0020C00F00203057050066
:104E8000E0120020704700BF034A0123118803FA93
:104E900000F0084310807047F01A002004490122F6
:104EA0000B8802FA00F023EA00030B80704700BF72
:104EB000F01A0020034B1B8843FA00F000F00100B9
:104EC000704700BFF01A0020F8B5114E114D124B7B
:104ED000124A134C1349144802273760134E2E60B0
:104EE000134D1D60102303251560236040F24652C8
:104EF0004FF4FA640F4D0B60026011460E482C60AF
:104F0000224600F061FB0D4B4FF6FF721A80F8BD90
:104F1000B80F0020C00F0020E0120020F41A00207B
:104F2000D0100020EC120020C40F002028810100C6
:104F3000D0967349043D00203C720020F01A0020F6
:104F4000DFF83CC0F0B40D4CDCF80030049E636028
:104F500081B1B6104F0033440022A1686360091587
:104F6000551C20F81210AAB2BA4219463344F4DB99
:104F7000CCF80010014BF0BC9B687047000C02405D
:104F80009C0600202DE9F843124E13483168089F13
:104F90004160D2B102F1FF381FFA88F803EB8808AC
:104FA0001C1F814600E03168D9F80850394431604F
:104FB000C9F8041054F8041F28B2FFF7C7FE2814DC
:104FC0002168FFF7C3FEA045EDD1034B9B68BDE808
:104FD000F88300BFA0060020000C024030B40A4D48
:104FE000043A011F00F1FC0451F8040F2B6803FB85
:104FF00000F3002BB8BF03F6FF7304321B13A1426A
:105000001360F1D130BC7047083D002092B1013AE5
:1050100092B230B403EB82020438043B0439002519
:1050200053F8044F40F8044F934241F8045FF7D11E
:1050300030BC7047704700BF2DE9F04F0C4C0D4D50
:1050400024686C60ADF65C0DCDE91423099100294C
:1050500000F0CA81821E069216AA002312920DF554
:105060008B6211930C95089313929B4606E000BF48
:10507000AC090020000C0240C74B1C68DDF88038EA
:105080000698C64F30F8022FC54E1C440C9B9968F9
:105090000690C14804605C60C24BA2F580521B7848
:1050A00008B2091402FB00F01BF0010F02FB01F231
:1050B00047F8230046F8232000F06481A3F10E0294
:1050C00002F03F0203F03F0457F8221056F8220086
:1050D000B54A1268029257F8242056F824400E94DC
:1050E000B14C2646A468009434690494D6E906E4D9
:1050F000AE4E079496F800A0029E9D1E86FB018985
:1051000005F03F05A64E57F8251056F825500F9587
:10511000A3F10C0404F03F04A3F1040C57F824504D
:105120000A95029D56F82470009EA3F10A04C5FB5F
:10513000028904F03F020E9C0D92C6FB018985FB9B
:1051400000010CF03F0CC5FB0401954D934E55F842
:105150002C400E940F9C009D56F82C60A446C5FB75
:105160000C012C46C4FB07019A1F02F03F020A9D66
:105170008A4FCDE90A010D988949A3F1080CC5FBB6
:1051800004890CF03F053C4657F820C051F8200038
:1051900057F8227051F82210049A0D97C2FB068925
:1051A000109146464F460E990F90DDE90A89084650
:1051B000073BCCFB0267C2FB008903F03F031046AC
:1051C000774A54F825C054F82340CDE90489B946FC
:1051D00052F8257052F82350DDE90412034604907A
:1051E0000F98C3FB0012B0461346109E0A460D9955
:1051F000CEFB0623CEFB0189CEFB07234046079F4B
:105200004946CCFB0E01C7FB0401C7FB0523D20FA7
:10521000C50F45EA410542EA43020899644B6548D7
:1052200043F82A50CB0740F82A2040F1A380AAF186
:105230000E020AF01F035E4950F823C051F82340C4
:1052400002F01F02AAF1020551F8227050F8222044
:105250005749029805F01F0580FB078951F8257012
:105260005449AAF10C0351F825100D9103F01F03C6
:105270004F4951F823100A914E4951F823500E9589
:1052800080FB0223CCFB0023AAF10406CDE9022314
:1052900006F01F06474A464BAAF10A0553F8263086
:1052A000C4FB008905F01F05009852F82640404EC7
:1052B000C7FB008956F825C052F825500A9A0F9569
:1052C000DDE902670D9DC2FB00890E9AC5FB0067F0
:1052D000C2FB00670498364AAAF1060101F01F01DB
:1052E000C3FB0089324BAAF10805CDE9006705F040
:1052F0001F0553F821602F4B53F8217052F82510E9
:105300000291DDE90012C4FB001253F82550134648
:105310000A460F99AAF1070AC1FB00230AF01F0AE7
:10532000234951F82A402349CCFB008951F82A002F
:105330000299C6FB0E89C1FB0E89C7FB0E23079994
:10534000C5FB0E23C4FB01891C461346C0FB013478
:10535000DA0F42EA4402129C11984FEAD8712546AE
:1053600041EA490145F820101399431C9BB241F8CA
:10537000202011931F210D48FFF7E2FC089B013309
:105380009BB208933F210748FFF7DAFC0BF10103BA
:105390001FFA83FB10E000BFAC09002024070020A7
:1053A000A4080020A509002068000020A40900200E
:1053B000A406002024080020099B5B457FF45CAE16
:1053C000149A12990B484FF4807301F089FC159AD6
:1053D000139909484FF4807301F082FC074B9B68D6
:1053E0000DF65C0DBDE8F08F16AB12930DF58B63D7
:1053F0001393E5E7386900202C690020000C024077
:10540000C2B1F0B4571EBFB200EB870704390438AD
:105410001E1F51F8044F50F8042F84FB04456C10F4
:1054200082FB022304EB6304874246F8044FF0D169
:10543000F0BC7047704700BF2DE9F04FDFF898B01F
:10544000234FDBF800407C6083B0002A3BD002F1A0
:10545000FF3A1E461FFA8AF300EB8303DFF87CA0B5
:105460001C4A0193051FA1F10408B94601E0DBF8CD
:1054700000400C9B00921919D9F80840CBF8001095
:10548000C9F80410DAF8000055F8041F27B24001EB
:1054900007FB00F0FFF75AFC0746DAF8000058F85F
:1054A000041F2414400104FB00F0FFF74FFC009A96
:1054B000019B116802290CBF3F183F1A9D423760BB
:1054C00006F10406D3D1024B9B6803B0BDE8F08F10
:1054D000000C0240B80F0020B0090020D0100020BE
:1054E00030B40A4D043A011F00F1FC0451F8040FD6
:1054F0002B6803FB00F3002BB8BF03F6FF730432E5
:105500001B13A1421360F1D130BC7047D0100020B2
:105510001B4B10B51B685A1E012A82B01AD91BB149
:10552000032B01D002B010BD164B17484FF4807406
:10553000CDE900340422154B802101F0B5FB144B5A
:105540001448CDE900340422104B802101F0ACFB5B
:1055500002B010BD0B4B0C484FF48074CDE9003401
:1055600004220D4B802101F09FFB094B0948CDE936
:1055700000340422084B802101F096FB02B010BDDC
:10558000B80F00202063002038690020A40200200A
:10559000446900202C690020A400002000B583B0DD
:1055A00040230093044A054B0548802101F0EEFB9F
:1055B00003B05DF804FB00BF3C720020406F002088
:1055C0001C690020000000002DE9F0410546ADF502
:1055D000826D50001C460E46FEF708FA1CA3D3E964
:1055E0000023FEF77DFACDE900017000FEF7FEF919
:1055F00017A3D3E90023FEF773FA9DED001B41ECDE
:10560000100B022202A8802100F0D6FBA008FEF7B2
:10561000FDF9022241EC100B02A8802100F0B0FE3F
:105620000DA7D7E90067043D02AC0DF5816832464D
:105630003B46F4E80201FEF753FAFEF701FDA045F0
:1056400045F8040FF3D10DF5826DBDE8F08100BF80
:10565000CA2E96E5AAF7073F0000C0FFFFFFDF4113
:1056600010B5094C82B001AB224601F0E5FB074AB8
:10567000236811689B128B42236003D008201360BB
:10568000FFF702FC02B010BDA80900202869002025
:1056900038B5094C094B2288094D0A4900EB4000F6
:1056A00003EB0013A8185D6ADA7B2B68FAF7ECFFAE
:1056B00023881844208038BDBC0F0020A40400209B
:1056C000B80D0020A4B1000838B50B4A0B4C0C4DA6
:1056D00021880C4B00EB400002EB00126818516A65
:1056E000D27B0D68084903EB8503FAF7CDFF2388C9
:1056F0001844208038BD00BFA4040020BC0F002047
:10570000B80D002058060020ACB100082DE9F04388
:105710002C4B2D4900EB400003EB001389B05B6A72
:1057200068461A68FAF7B0FF9DF80090B9F1000FCB
:1057300045D00025254F2C462E464FF02E086846B2
:10574000FAF7DEFF001BA7FB00235B0803EB430314
:1057500098420CD108AB1E444CB116F8213C202BCA
:1057600028D008AB2B4403F8108C0135EDB201347E
:10577000E4B208AA08A96B1C22440D44264605F889
:10578000109C12F8209CDDB2B9F1000FD7D1104C5B
:1057900010482288104908AB1D441044002304AA75
:1057A00005F8103CFAF770FF23881844208009B0F0
:1057B000BDE8F08308AA2A4402F8103CD5E74D461C
:1057C000E5E700BFA404002098B10008ABAAAAAA8C
:1057D000BC0F0020B80D0020A0B10008F8B5184B90
:1057E00000EB400003EB001000AFC17B426ACB1D11
:1057F00003F4FC73ADEB030D68461378E1B14D1E65
:10580000EDB201356D446C464FF0200C852609E061
:1058100026709A1F0134D2B29A4294BF13460023D5
:10582000A54209D0052BF3D8A3F180020BB1227059
:10583000EFE784F800C0ECE7FFF7B0FABD46F8BD2B
:10584000A40400202B38F8B5362854D8DFE810F02F
:10585000640053007F005300530053005300530073
:1058600053005300530053005300530053005300A0
:10587000530053005300530053005300A300530040
:1058800053005300460037005400A900DF005300C6
:105890005300530053005300530053005300530070
:1058A0005300530053005300530053005300530060
:1058B000530053005300530053005300EE005E4B5F
:1058C0005E4A1B7803EB430302EB03125369D16971
:1058D00003EB83035B008B4200D25361584B594D5D
:1058E000594C2A8803CB1E88131902F109072F800F
:1058F000105159601E81F8BD4F4B504A1B7803EB85
:10590000430302EB03135A69092AE7D94F49A1FB64
:105910000212D2085A61E1E7474C484D2078420014
:10592000131805EB03135E6A5F693168394431600F
:105930009F69B94202D3DB69994222D9024405EB3F
:10594000021292F82030DBB9D369336019E03A4C87
:105950003A4D20784200131805EB03135E6A5F6925
:105960003168C91B31609F69B94202D3DB69994232
:1059700007D9024405EB021292F82030002BE3D144
:105980003760FFF781FA237803EB430305EB031538
:10599000AB6A9847A2E7FEF721FEBDE8F840FEF7A4
:1059A000BDBD254C2078FFF76FFA2078284B0138D1
:1059B0001B78C0B29842207002D3581EC0B220702B
:1059C000204D214EFFF760FA28882249002301224A
:1059D0003044FAF759FE28882278184B1E49841D56
:1059E000A4B202EB420003EB001330192C80FAF74B
:1059F0004BFE2B88124A034403CA9BB29C1903F145
:105A000009072F801288985161602281F8BD0A4CE5
:105A10002078FFF739FA20780D4B01301B78C0B29F
:105A2000834220709CBF00202070C9E7FEF796FDDE
:105A3000BDE8F840FEF7AABD3D740020A404002094
:105A4000A8B00008BC0F0020B80D0020CDCCCCCCF5
:105A500054060020B4B00008C0B00008F8B50F4DDF
:105A60000F4E28880F4F104900242346012230444E
:105A70003C70FAF709FE2C883A780C4B0C49063436
:105A8000A4B202EB420703EB071330192C80FAF79C
:105A9000FBFD2B8818442880F8BD00BFBC0F0020F8
:105AA000B80D00203D740020B4B00008A40400200C
:105AB000C0B00008F8B50E4D0E4E28880E490023E0
:105AC00001223044FAF7E0FD0C4B2C881A780C4B7D
:105AD0000C490634A4B202EB420703EB071330195A
:105AE0002C80FAF7D1FD2B8818442880F8BD00BF20
:105AF000BC0F0020B80D0020B4B000083D74002099
:105B0000A4040020C0B000082DE9F843224E3378E9
:105B1000002B39D0DFF89890204FDFF898800024D0
:105B200004E001343378E4B2A3422DD92046FFF7D4
:105B3000C1F90028F5D065002A1909EB021238884E
:105B4000137C1749527C4044FAF79EFD3B88154A66
:105B500015491278184480B2431CA2429BB215D05A
:105B60000A8820F808203B80254409EB05152046CB
:105B7000AB7B0BB9EB6A98472046FFF78FF90134EE
:105B80003378E4B2A342D1D8BDE8F883074A3B801A
:105B9000138820F80830E7E754060020BC0F0020E7
:105BA000B4B000083D7400200CB2000894B10008A5
:105BB000A4040020B80D0020DFF8C8C12DE9F84387
:105BC000BCE80F00DFF8C081634CB8F80050634EAA
:105BD000285105EB040EDCF80000CEF80410CEF8D6
:105BE0000820CEF80C30CEF810000FCE9CF804C080
:105BF0008EF814C005F1140E1FFA8EFE0EEB040C85
:105C0000574F4EF804003068CCF80410CCF8082048
:105C1000CCF80C30CCF810000FCF05F12A0EB6F8F6
:105C20000490B679ACF814901FFA8EFE8CF81660CA
:105C30000EEB040C4EF80400CCF8041003CF494ED0
:105C4000CCF80820CCF80C30CCF81000CCF81410AC
:105C50000FCE05F1420E1FFA8EFE3F788CF81870B9
:105C60000EEB040C4EF80400CCF8041003CE3E4FAB
:105C7000CCF80820CCF80C30CCF81000CCF814107C
:105C80000FCF05F15C0E1FFA8EFEB6F80090B678C5
:105C90008CF81A60ACF818900EEB040C4EF8040067
:105CA000CCF80410CCF80820CCF80C3007CF2F4EDD
:105CB000CCF81000CCF81410CCF818200FCE05F159
:105CC000780E1FFA8EFE3F788CF81C700EEB0407DE
:105CD0004EF804007960BA6007CE9635B6F800C079
:105CE000B6783861ADB27961BA61FB60A7F81CC0C3
:105CF000BE7760191E49A8F8005047F23052FAF7F3
:105D0000C3FCB8F800301B4A03F1080503CAADB262
:105D10002E19123328519BB2957817887160B5728D
:105D2000E018154937810022A8F80030FAF7ACFCDA
:105D3000B8F800301149124A0E881588181D591DEF
:105D40009A1D80B289B292B207330653A8F8003088
:105D50000D531553BDE8F883B80D0020E4B00008DA
:105D6000FCB0000818B1000834B1000854B10008B4
:105D700074B100087CB1000888B10008B0B1000817
:105D800090B10008CCB00008BC0F0020074BF0B465
:105D9000074D084C2A8803CB1E881051131902F1B5
:105DA000090759601E812F80F0BC7047A8B0000819
:105DB000BC0F0020B80D00202DE9F04F2DED048B15
:105DC0008DB081468B468DED000B042A18D8DFE894
:105DD00012F01C006700CF004F010500002903DD11
:105DE000CA000021FAF71EFB0BF1FF3B0BEBDB7B3C
:105DF000CB4B4FEA6B0B002209EBCB09C9E900231F
:105E00000DB0BDEC048BBDE8F08F0029F8DD481E15
:105E1000FDF7FCFD0022C34BFDF762FEB6A3D3E9FC
:105E2000002304460D46DDE90001FDF759FE4FF061
:105E30000008CDE90201DA460CE030463946FEF7AB
:105E4000C1F8F0B1DDE9000108F10108C245E9E857
:105E50000201D5D04046FDF7D9FD22462B46FDF77D
:105E600087FCDDE90223FDF73BFEA5A3D3E9002370
:105E700006460F46FEF7C4F8A3A3D3E90023002883
:105E8000DBD147EC106BFBF7DFF932463B4651ECB8
:105E9000100BFDF74FFFDDE90023FDF721FED3E7EF
:105EA000002901F00103B8BF5B42012B00F0D38150
:105EB0000029A5DD481EFDF7A9FD0022994BFDF73D
:105EC0000FFE8DA3D3E9002304460D46DDE9000152
:105ED000FDF706FE9FED8E9BCDE902014FF0000815
:105EE000DA4607E089ED009B08F10108C24509F197
:105EF000080985D04046FDF789FD22462B46FDF76F
:105F000037FC0022002306460F46FEF751F83246C2
:105F10003B460028E6D1DDE90201FDF7E1FD41EC59
:105F2000100BFBF731F974A3D3E90023B0EE408ADC
:105F3000F0EE608A30463946FDF7D2FD41EC100B99
:105F4000FBF722F974A3D3E9002351EC180B8DED74
:105F5000000BFDF7C5FD32463B46FDF7EBFE9DED20
:105F6000000B53EC102BFDF705FCC9E90001BBE762
:105F700051EC110B00226B4BFDF7B2FDDDE9006720
:105F800004460D4602460B4630463946FDF7F0FB07
:105F90003246CDE900013B4620462946FDF7EAFBA3
:105FA000BBF1000F04460D467FF72AAF0BF1FF301F
:105FB000FDF72CFD00225B4BFDF792FD4EA3D3E9CC
:105FC000002307468846DDE90001FDF789FD4AA365
:105FD000D3E90023CDE9000120462946FDF780FDE5
:105FE0009FED4B9BCDE902010026DA4607E089EDE3
:105FF000009B0136564509F108093FF401AF3046D0
:10600000FDF704FD3A464346FDF7B2FB00220023AC
:1060100004460D46FDF7CCFF22462B460028E6D16C
:10602000DDE90001FDF75CFD41EC100BFBF7ACF87E
:1060300022462B46DDE90201B0EE408AF0EE608A8E
:10604000FDF74EFD41EC100BFBF79EF851EC180BE1
:1060500053EC102BFDF78CFB2FA3D3E90023FDF7A6
:106060003FFD22462B46FDF765FEC9E90001C0E76A
:1060700051EC110B00222B4BFDF732FDDDE90067DF
:1060800004460D4602460B4630463946FDF770FB86
:106090003246CDE902013B4620462946FDF76AFB20
:1060A000BBF1000F04460D46CDE904457FF7A8AECD
:1060B0000BF1FF30FDF7AAFC00221A4BFDF710FD93
:1060C0000DA3D3E90023CDE9060120462946FDF7BB
:1060D00007FD09A3D3E90023CDE90801DDE90201A9
:1060E000FDF7FEFC4FF0000ACDE90A01CDF8009063
:1060F0006BE000BFAFF30080182D4454FB21094032
:10610000F168E388B5F8E4BEF168E388B5F8E43EE9
:10611000000000000000000083C8C96D305FD43F5C
:106120000000F03F0000E03F8FA3D3E900232046AA
:106130002946FDF747FF00285ED08F4F00264246D4
:106140004B46DDE90801FDF7CBFC85A3D3E900232D
:1061500004460D46FDF754FF00286BD082A3D3E917
:10616000002320462946FDF72DFF002862D0DDE9F7
:10617000042330463946FDF7FBFA42464B460646B5
:106180000F46DDE90A01FDF7ABFC75A3D3E9002357
:1061900004460D46FDF734FF00283AD072A3D3E938
:1061A000002320462946FDF70DFF90B3DDE90223C9
:1061B00030463946FDF7DCFA009BE3E802010AF1BC
:1061C000010AD34500933FF41BAE5046FDF71EFC79
:1061D000DDE90623FDF7CCFA65A3D3E90023804669
:1061E0008946FDF77DFC5EA3D3E9002304460D46F6
:1061F000FDF706FF002897D145EC104BFBF724F87C
:1062000022462B4651EC100BFDF794FD06460F4637
:1062100095E745EC104BFBF717F822462B4651EC5F
:10622000100BFDF787FDDDE90223FDF759FC02465F
:106230000B46BDE745EC104BFBF706F822462B4614
:1062400051EC100BFDF776FDDDE90423FDF748FC6A
:1062500002460B468DE700297FF7D2AD481EFDF7B9
:10626000D5FB0022454BFDF73BFC41A3D3E90023BE
:10627000CDE90201DDE90001FDF732FC4FF0000835
:10628000CDE90401CDF818B02FE020462946FDF7EE
:1062900099FE002843D0DFF8E0B04FF0000ADDE9B6
:1062A000042330463946FDF71BFC2DA3D3E9002318
:1062B00004460D46FDF7A4FE2BA3D3E900230028D6
:1062C0003AD020462946FDF77DFE002834D0DDE98E
:1062D000002350465946FDF74BFA069B08F101088A
:1062E0009845E9E802013FF48BAD4046FDF78EFB8F
:1062F000DDE90223FDF73CFA1DA3D3E9002306469E
:106300000F46FDF7EDFB16A3D3E9002304460D4627
:10631000FDF776FE14A3D3E900230028B5D145ECA0
:10632000104BFAF791FF22462B4651EC100BFDF76C
:1063300001FD82468B46B2E745EC104BFAF784FF2D
:1063400022462B4651EC100BFDF7F4FCDDE900234F
:10635000FDF7C6FB02460B46BBE700BFAFF300806C
:10636000F168E388B5F8E4BEF168E388B5F8E43E87
:10637000182D4454FB2109400000F03F0000E03F8D
:10638000012A00F013822DE9F04F2DED048B0B460E
:106390008FB00233DB000C90184657EC106B059160
:1063A00015460893F9F794FF0490002800F08D80BB
:1063B0000022D74B30463946FDF70EFE002800F08C
:1063C0008180002200233046394647EC186BFDF7E8
:1063D0000DFE002873D0059B581CFDF717FB022DFE
:1063E000CDE9060176D0032D00F0E1810E2D5ED1BE
:1063F000059B03EBD37A4FEA6A0ABAF1000F42DD3C
:1064000002460B460020C349FDF794FCB6A7D7E926
:106410000067DDF8109004460D46C8464FF0000BAB
:106420000BF1010B5846FDF7F1FA32463B46FDF7FA
:1064300057FB22462B46FDF753FB41EC100BFAF7B6
:1064400003FFD345A9EC020BEAD1049B03EBCB0479
:1064500098ED000BB0EE481AF0EE681AFAF754FF08
:10646000A8EC020B4445F3D1089B103B0993099B10
:10647000049A194611440023F2E8024501335B45B2
:1064800061E90245F8DB059B002B10DD089B103B02
:1064900009930C9C049D23441E46D4E90001F5E8B1
:1064A0000223FDF71DFBE4E80201A642F5D10498A2
:1064B0000FB0BDEC048BBDE8F04FF9F711BF9FEDB5
:1064C0008C8B88E70026924F7BE70FB0BDEC048BE6
:1064D000BDE8F08F059B03EBD37B002B4FEA6B0BE2
:1064E00040F3C58102460B4600208A49DFF824921A
:1064F000FDF720FC0022CDE90A01874B51EC180B77
:10650000FDF7EEFA089B049ACDF834B0103B0993DE
:10651000D3184FF0000841EC180B039392462F4616
:1065200079E0022E00F0FF80032E00F00781042E98
:1065300000F01081052E00F01981062E00F01C815C
:10654000072E00F02581092E40F0BB806AA3D3E915
:106550000023FDF7C5FA02460B46FDF7C1FA0246D5
:106560000B4620462946FDF705F942464B46FDF706
:1065700001F9CDE900014FF0010B00240025584638
:10658000FDF744FAB0EE480AF0EE680A41EC110B50
:10659000FAF7BAFEBBF1010F51EC100B00F082804C
:1065A000BBF1020F00F0BA80BBF1030F00F0C08016
:1065B000BBF1040F00F0C880BBF1050F00F0D080E4
:1065C000BBF1060F69D0BBF1070F00F0DB80BBF118
:1065D000090F7ED148A3D3E90023FDF781FA0246D3
:1065E0000B46FDF77DFA02460B4620462946FDF78D
:1065F000C1F842464B46FDF7BDF80B460246DDE9C1
:106600000001FDF797FBEAE80201039B534507F100
:10661000020700F0C3803846FDF7F8F9DDE90623EC
:10662000FDF7A6F8DDE90A23FDF75AFA02460B4604
:10663000FDF756FA02460B4640464946FDF798F8E4
:1066400041EC100BFAF7FCFF53EC182B51EC100B3C
:10665000FDF746FA41EC190B0126002400253046CF
:10666000FDF7D4F9B0EE490AF0EE690A41EC110BDE
:10667000FAF74AFE012E51EC100B7FF452AF02469E
:106680000B46FDF72DFA02460B4620462946FDF73C
:1066900071F8013604460D46E1E719A3D3E900235A
:1066A000FDF71EFA02460B46FDF71AFA02460B46A4
:1066B00020462946FDF75EF80BF1010B04460D4616
:1066C0005DE711A3D3E90023FDF70AFA02460B4662
:1066D000D7E70DA3D3E90023FDF702FA02460B46E4
:1066E000E2E700BFAFF30080182D4454FB210940BE
:1066F000000000000000000034C756A5E31DC73E9F
:10670000176CC1166CC1563F1AA0011AA001FA3EBF
:10671000000024400000F03F0000E03F0022664BF4
:10672000FDF7DEF9BEE70022634BFDF7D9F9A6E7D6
:1067300051A3D3E90023FDF7D3F9B3E74EA3D3E97F
:106740000023FDF7CDF99AE74DA3D3E90023FDF728
:10675000C7F9A7E74AA3D3E90023FDF7C1F98EE7FC
:1067600049A3D3E90023FDF7BBF99BE746A3D3E98F
:106770000023FDF7B5F982E745A3D3E90023FDF730
:10678000AFF97CE744A3D3E90023FDF7A9F989E732
:1067900041A3D3E90023FDF7A3F970E7DDF834B096
:1067A000BBF1000F3FF763AE099B72E67047059B94
:1067B00003EBD37B002B4FEA6B0B58DD089A04994F
:1067C000CDF800B0103A099201EB0209C3F10108BB
:1067D0000D460C46DDE906AB0CE030463946FDF7C8
:1067E000F1FB28B335490020E4E80201A14508F196
:1067F00002082DD052465B4629A1D1E90001FDF7E0
:1068000099FA064640460F46FDF700F902460B4648
:1068100030463946FDF764F923A3D3E90023064641
:106820000F46FDF7EDFB22A3D3E900230028D4D1C6
:1068300047EC106BFAF708FD32463B4651EC100B63
:10684000FDF778FAE4E80201A14508F10208D1D188
:10685000DDF800B0B0EE481AF0EE681A95ED000BC6
:10686000FAF752FDA5EC020BAC42F3D198E7BBF16D
:10687000000F7FF71CAEF7E5555555555555C53FEB
:10688000555555555555A53F111111111111813F00
:10689000176CC1166CC1563F1AA0011AA0012A3FFD
:1068A000182D4454FB210940F168E388B5F8E4BE93
:1068B000F168E388B5F8E43E0000E03F0000F03FF7
:1068C000FEE700BFFEE700BFFEE700BFFEE700BF38
:1068D000FEE700BF704700BF704700BF704700BFB2
:1068E00001F04ABB014802F031BB00BF700C002030
:1068F000014802F02BBB00BF740A0020014802F0DF
:1069000025BB00BFB4090020014802F01FBB00BF37
:10691000100B0020014800F069BC00BF700B002084
:10692000014803F087BB00BFDC0B0020014803F0E7
:10693000ADB800BF4C0D00200B4B1A6E42F00102A7
:106940001A661A6E82B002F001020092009A9A6DE5
:1069500042F080529A659B6D03F080530193019B36
:1069600002B002F0C1BB00BF001002400368B3F1E7
:10697000A04F00D0704703F1704303F5043370B5A6
:10698000DA6C184C184942F40052DA64DB6C21606E
:1069900082B003F40053019305224FF4807305463F
:1069A00080204FF480616260206120226361204674
:1069B0000023019E2362C4E90612C4E9023302F0F7
:1069C00059F960B900226C6511461220A56202F0E7
:1069D000A5FB122002B0BDE8704002F0D5BBFEF767
:1069E000ADF9EFE7700C00200800024002680A4B86
:1069F0009A4200D07047D3F8482442F00802C3F806
:106A0000482403F5806382B09B6C03F00803019374
:106A1000019B02B0704700BF000C024070B50268D5
:106A2000334B88B000249A42CDE90344CDE90544B4
:106A3000079401D008B070BD03F1704303F5023331
:106A40002C4DDA6C42F48032DA64DA6C02F4803273
:106A50000192019ADA6C42F00102DA64DB6C03F015
:106A6000010302933022032303A9064602980392EE
:106A70004FF09040049302F011F81F49296006225C
:106A8000102380204FF400716A60AB604FF4006205
:106A9000202328612846EC602C62C5E90512EB61D1
:106AA00002F0E8F8E8B9154C154B236007211022D5
:106AB00080204FF40073B5606160A2604FF4006104
:106AC00020222061636120460023AE62C4E90612E1
:106AD000E360236202F0CEF830B9F460A66208B039
:106AE00070BDFEF72BF9DEE7FEF728F9F5E700BFEA
:106AF00000080050740A00201C000240B409002065
:106B00004400024010B50168114A86B0002391424A
:106B1000CDE90133CDE90333059301D006B010BDB3
:106B200003F1804303F5043301A9DA6C42F001025A
:106B3000DA64DB6C03F0010300930A2203234FF0B5
:106B40009040009CCDE9012301F0A8FF06B010BDE4
:106B50000003014000B503681D4A934285B015D07B
:106B60001C4A93421FD01C4A934202D005B05DF8E4
:106B700004FB1A4B1A6E42F400521A661B6E03F4A1
:106B800000530393039B05B05DF804FB134B9A6D10
:106B900042F010029A659B6D03F010030193019B74
:106BA00005B05DF804FB0D4B9A6D42F020029A652A
:106BB0009B6D002203F02003029311463720029BB5
:106BC00002F0ACFA372005B05DF804EB02F0DCBA55
:106BD000001000400014004000340140001002404A
:106BE00070B50268264B88B000249A42CDE9034470
:106BF000CDE90544079401D008B070BD03F55843B2
:106C0000204D1A6E42F480421A661A6E02F48042D7
:106C10000192019ADA6C42F00102DA64DB6C03F053
:106C2000010302934FF4C063022203A903930646B3
:106C30000723029804924FF09040079301F02EFF33
:106C4000114828601921102280232846EC60C5E9EC
:106C50000544C5E90744C5E901122B6102F00AF8B1
:106C600058B900221146B5672520AE6202F056FAE7
:106C7000252002F089FA08B070BDFEF75FF8F0E752
:106C800000380140100B002058000240054BD3F89B
:106C900088204FF0006142F47002C3F888209960A8
:106CA000704700BF00ED00E0F8B5DDE9067CBCFBF5
:106CB000F2F402FB14C484B9164601F18042013A91
:106CC0000546624441804360920021463846F9F708
:106CD000A9FB2E70AF602046F8BD6FF00100F8BD33
:106CE0002DE9F04F85B08568B0F802C0029589465D
:106CF00001784068B3FBF1F4009103940190002CFB
:106D000042D00CF18043013B9B002046043B05EB45
:106D100003084FEA810E8246AB46009B4046494637
:106D200051F8044B40F8044F013BF9D1F14463465C
:106D3000BCF1000F0ED0019D5C460020002154F8EC
:106D4000047B55F8046B013BC6FB0701F7D1C30F69
:106D500043EA4103BAF1010AF34442F8043BF04428
:106D6000DBD1DDE9022303FB0E2EBCF1010C08D0C0
:106D7000029B043B5EF8042B43F8042FBCF1010C8A
:106D8000F8D105B0BDE8F08FAE46EEE738B5049C0B
:106D9000826004F18044013C0C4401800546A2005D
:106DA00018460021F9F73EFB686038BD2DE9F04F29
:106DB00083B04468B0F800C00094D0F808A00193F4
:106DC000C3B389460CF18041013989001846043962
:106DD00004EB010E8346A04659F8043B4EF8043FED
:106DE0005546634644460020002154F8047B55F87C
:106DF000046B013BC6FB0701F7D1C30F43EA410314
:106E0000BBF1010B08F1040842F8043BE4D1DDE9D1
:106E1000003203EB8202BCF1010C08D0009B043B62
:106E200052F8041B43F8041FBCF1010CF8D103B065
:106E3000BDE8F08F2246EEE70129F0B4066811D0D4
:106E4000051D0027012055F8044BA642B8BF074690
:106E500000F10100B8BF26468142F4D116601F60E0
:106E6000F0BC7047002716601F60F0BC704700BF81
:106E700070B582B000230193002800F0A380C56D97
:106E80000446002D00F09380226893689D0005D58C
:106E9000936823F0204323F03F0393609368D80066
:106EA00019D4764B76481B6891689B09A0FB0303B5
:106EB0009B0921F01041013321F03F015B0041F0BB
:106EC000805191600193019B2BB1019B013B019388
:106ED000019B002BF9D19368D9005AD4E36D43F09C
:106EE0001003E365236E43F001032366936813F0F8
:106EF000040F4FF00100E36D52D1DB0650D4E36D77
:106F000023F4817343F00203E3659368DE0709D439
:106F10004FF0A0435B499B688968CD0703F00103EC
:106F200040F18380D4E90215E36B2B430B43657F6B
:106F300094F8241043EA4533012943EA014303D17D
:106F4000A16A013943EA4143E16A21B1256B01F4A9
:106F5000787129430B43D6684B49656B31400B432D
:106F6000D360136923F040632B431361936859077F
:106F70002BD593686369012B4FD0136B23F00F035C
:106F80001363E36D23F0030343F00103E36502B0F1
:106F900070BD936813F0040F4FF00000E36DACD0A8
:106FA000E36D012043F01003E36502B070BDFFF70D
:106FB000DDFC22682566936884F858509D007FF5B3
:106FC0006DAF65E7012002B070BD93681B07D1D497
:106FD000D16894F83830267F256921F480415B0020
:106FE00021F0020143EA86330B43D36013693DB3BA
:106FF00043F480331361D2F8C03023F47F5323F07D
:107000003F032B43C2F8C03094F84030012B23D00B
:10701000136923F001031361ACE7116B236A21F0BC
:107020000F01013B0B431363ABE7002B7FF47AAFF7
:10703000164965688B6823F47C132B438B6071E7DA
:1070400023F480331361D2F8C03023F47F5323F04C
:107050003F03C2F8C030D7E7D4E91131E66C256DA3
:107060000B43116943F00103334321F4FF612B43C8
:1070700021F004010B4313617CE700BF6806002088
:10708000632D3E05000100500740F0FF0003005053
:107090002DE9F047494B06689D68B3685C0728D422
:1070A00090F85830012B24D005F01F050123092D3D
:1070B00090460F46044680F8583005D9002384F8DE
:1070C00058300120BDE8F08740F22123EB40DB0778
:1070D000F4D5B368D8070FD4B268394B1A4247D0F9
:1070E000E36D43F01003E365236E43F00103236671
:1070F000E4E70220BDE8F087E36D324A23F47063D1
:1071000023F0010343F480739642E36552D0E36DAC
:1071100023F48013E365E36D606D2B492B4A13F470
:1071200080531CBF236E23F006032366284BC362E3
:107130001C23C0E90C1233607368002243F0100373
:1071400084F858207360F16841F0010143463A46E3
:10715000F16006F1400101F025FE2268936823F0FA
:10716000004323F03F0343F004039360BDE8F0873E
:10717000B368184A134043F00103B360924600F02D
:1071800007FF266881463368DB07B5D4B368D907A3
:1071900005D4B36803EA0A0343F00103B36000F0C7
:1071A000F7FEA0EB090002282668ECD93368DA075D
:1071B000E9D495E7002DAAD0ADE700BF0003005049
:1071C0003F00008000010050DD710008A574000838
:1071D0003D740008C0FFFF7F704700BF08B5806A9C
:1071E000FFF7FAFF08BD00BF704700BFF8B503689E
:1071F000904A1D685E689768A907044607F01F0754
:1072000002D5B20700F1A18069077BD5720779D555
:10721000E26DD20603D4E26D42F40072E265DA68F0
:1072200012F4406F1CD1844A934200F0DF80DA6888
:10723000900415D41A68110712D59A68520700F104
:10724000E6805A6822F00C025A60E36D23F48073E2
:10725000E365E36DDB0403D4E36D43F00103E36511
:107260002046FDF7EBF823680C221A60A8064FD5DC
:10727000B1064DD5E26DD10603D4E26D42F4005261
:10728000E2656D48DA6CD968834202F4C07201F499
:10729000406168D0D868D2B9820100F1A0801A6834
:1072A000520614D5810212D49A68120700F1B880F0
:1072B0005A6822F060025A60E36D23F48053E3655C
:1072C000E36DD80503D4E36D43F00103E365204685
:1072D00000F0A0FD236860221A60290601D532065D
:1072E00066D4E80501D5F1056DD4AA0501D5B00530
:1072F00052D4E90601D5F2060FD4680501D571050F
:107300003AD4F8BD2807B1D5310781D4A806AFD447
:107310006A06E2D57006E0D5ACE7E26B32B1002F29
:1073200071D0444A926812F4604F0BD0E36D43F47D
:107330008063E365236E43F0020323662046FFF774
:1073400053FF236810221A60D7E7C36DD80603D411
:10735000E36D43F40063E365204600F063FD2368BA
:1073600002221A6050E7002F94D0B81F012891D94B
:107370004FF0A040C0688EE7E26D42F48042E265C3
:10738000226E4FF4806142F00802226620461960A6
:10739000BDE8F84000F040BDE36D43F48023E365B1
:1073A000204600F03DFD23684FF400721A60A0E70C
:1073B000E36D43F48033E3652046FDF749F8236825
:1073C00080221A608DE7E36D43F40033E3652046C5
:1073D00000F024FD23684FF480721A6085E70029CD
:1073E0007FF475AF81043FF572AF58E7092F03D9D9
:1073F0004FF0A042D2681BE740F22122FA40D207A8
:107400003FF515AFF4E7DA68D7079BD58EE7E36D54
:1074100043F01003E365236E43F0010323661FE787
:10742000E36D43F01003E365236E43F0010323662D
:107430004DE700BF0003005000010050836ADA6D81
:1074400012F0500F10B5DA6D1DD1196842F40072B8
:10745000DA650A6812F0080FCA681BD012F4406F90
:107460000DD1CA6894040AD4DA6D22F48072DA6508
:10747000DA6DD10403D4DA6D42F00102DA65184600
:10748000FCF7DCFF10BDD20607D45B6DBDE81040F1
:107490005B6B18479007F2D4E6E71846FFF7A4FEA7
:1074A00010BD00BF806A08B5C36D43F04003C365DB
:1074B000036E43F004030366FFF796FE08BD00BFAA
:1074C0002DE9F041034682B093F858200020012AAC
:1074D000019000F011811A6894680120650783F813
:1074E00058004FD4D1E90004A60906F00C0602F1B9
:1074F000300504F01F0477594FF01F0C0CFA04FC00
:10750000C0F38460A04027EA0C07384370519068AC
:10751000440749D590680C689068C00713D4CE68BA
:10752000C748D2F8B050DFF840C306F01807F8405B
:10753000C4F31207204025EA070528436645C2F830
:10754000B00000F08B80BF490C422BD0BE4DBF492C
:10755000A8688C4200F0E0761ED0BD498C421BD05A
:10756000BC498C4240F0CC8010F080701AD1BA49EE
:107570008A4217D0AA6822F0E072164346F080765D
:10758000AE6003E0DA6D42F02002DA65002283F893
:10759000582002B0BDE8F081010203D4B2F1A04F3F
:1075A00000F0D3800020F1E795680C6815F008051D
:1075B000B2D18E68C4F3045E0720E40D00FA0EF029
:1075C000B6F1004F04F004046FEA000002F1140C5D
:1075D00000F0DA8054F80C7006FA0EF638400643D4
:1075E00044F80C60506920F000405061D1F810C0A0
:1075F000D7680C68BCF1040F02F1600000F0CE8087
:107600004E6950F82C80DFF864E2C7F3C1077F00B1
:1076100004F0F84444F00044BE40264308EA0E0E4D
:1076200046EA0E0640F82C600F698E6950F8274034
:1076300091F81CC024F08074344340F827400E6950
:1076400050F82640BCF1010F24F0007408BF4FF041
:107650000075254340F826500C685DE7002F63D085
:1076600094FAA4F0002800F02381B0FA80F00130F1
:1076700000F01F00092840F21B8194FAA4F00028B2
:1076800000F04181B0FA80F00130800600F0F8404F
:1076900094FAA4F5002D00F03B81B5FA85F501358B
:1076A00005F01F05012606FA05F5284394FAA4F40F
:1076B000002C00F02B81B4FA84F4013404F01F0490
:1076C00004EB44041E3C240544F000742043C70D21
:1076D00007F0040702F11405C0F304507C598E68CA
:1076E0004FF0070C0CFA00FC24EA0C0406FA00F038
:1076F000204378510C6826E7022002B0BDE8F081F3
:1077000056498C427FF44EAF10F480007FF44AAFAC
:1077100051498A423FF446AFAA6822F0E0723243F0
:1077200042F48002AA6031E7A40E013404F01F0580
:10773000A0060124AC4000F0F840092D40EA040006
:1077400005EB4504BED82405C0E73F48444A81689C
:10775000444C21F0E0710E4346F400068660126846
:107760009209A4FB02129209013202EB420292003A
:107770000192019A002A3FF415AF019A013A019251
:10778000019A002AF9D10DE754F80C60304044F812
:107790000C00506940F00040506127E7156E156EEF
:1077A000C4F31207C5F38465002F41D1C4F3846686
:1077B000B54206D1146E24F0004414660C68C4F37C
:1077C000120745684668C6F38466002F50D1C4F39B
:1077D0008465AE4240F09E80446824F000444460DA
:1077E0000C6885688668C4F31205C6F38466002DAC
:1077F00049D1C4F38465AE4200F10C0740F08F809C
:10780000846824F0004484600C6838683868C4F3E5
:107810001205C0F38460002D42D1C4F38465854213
:107820007FF47AAE386820F0004038600C6873E668
:1078300094FAA4F6002EC4D0B6FA86F6B8E700BFD4
:10784000FFFF07000000088000030050000021C374
:107850001000C090000052C700010050000084CB0F
:1078600068060020632D3E0500007F4000F0FF0306
:1078700094FAA4F51DB1B5FA85F5AE42ACD0856891
:107880008668C6F3846694FAA4F58DB3B5FA85F5D7
:10789000AE4200F10C07B3D038683868C0F384609A
:1078A00094FAA4F5002D3FF437AEB5FA85F5B6E7A6
:1078B00094FAA4F020B3B0FA80F00130800600F012
:1078C000F84094FAA4F5CDB1B5FA85F5013505F087
:1078D0001F05012606FA05F5284394FAA4F454B1CD
:1078E000B4FA84F4013404F01F0404EB44042AE7DE
:1078F00000F10C07D0E74FF44014E7E60225EBE770
:107900004FF08060DDE74FF08060C1E6064CDDE6B9
:107910000225CAE686688668C6F384666BE7C66891
:10792000C068C0F384607AE7000050FE90F85830D9
:10793000012B00F0A680F0B404680B68A2684F68C1
:10794000012680F8586056071D4637D5A368B74A08
:107950009542D1E904635AD0E26802F01802182A6D
:1079600000F09280E268C2F3C102C2EBC271E26829
:107970004900043102F0180201F01F01182A26FA0A
:1079800001F100F08980E268C2F3C102C2EBC27269
:107990005200043202F01F02D340AD0C05F00C057A
:1079A000203443EA01432A5902F0F0221343002213
:1079B0002B5180F85820F0BC10467047A26812077F
:1079C000C5D49A4A93422ED0B7F1807F00F0A980A7
:1079D00064D9B7F1C07F00F0A480B7F1E07F02D096
:1079E000B7F1A07F60D1924E8A68B342C2F312050C
:1079F00000F0B180002D40F0CD80C2F384620125FB
:107A00009540D4F8A4202A43C4F8A42064E0E16897
:107A1000E268C1F3C101C2F3C1024900520006FA93
:107A200001F19340B9E7B7F1807F00F0BC8065D9E0
:107A3000B7F1C07F00F0CD80B7F1E07F00F0BC80EF
:107A4000B7F1A07F00F0CE80E36823F0FB4323F47E
:107A50008003E360236A8D690A7B23F4E0432B43B0
:107A60002362C36D802523F48033C365256063687A
:107A70000D68012A0CBF43F0800323F0800363608C
:107A800065E7022318467047E26802F01802182AD8
:107A90004FEA86017FF477AF9B007EE7B7F5000FD2
:107AA0003FD0B7F5400F9ED003F00102D5002A4425
:107AB000C3F3015505EB820504F10C0223F00246E5
:107AC00052F8253026F4601623EA060342F82530E2
:107AD000574A0B6893424AD0C26D0D7B22F4802234
:107AE000C2654FF4007222606268012D0CBF42F43F
:107AF000007222F400721D46626028E7B7F5000F9D
:107B00007DD0B7F5400F9FD1E2688B6822F0FB4231
:107B100022F4800203F0F843134343F44003E3608C
:107B200098E703F00102D6003244C3F3015606EB96
:107B3000820604F10C0523F0024C55F8262023F0B0
:107B40007E472CF4601C22EA0C0327F4F0073B4329
:107B500045F82630BCE7002D5AD1C2F384620123D8
:107B600003FA02F2D4F8A0301343C4F8A030C36D76
:107B70000A7B4FF4807523F40033C3652560636886
:107B8000012A0CBF2B4323F480736360D1E90463A3
:107B9000274DE1E692FAA2F2002A42D0B2FA82F22E
:107BA000012595402DE7E36823F0FB4323F4800390
:107BB00043F08073E3604DE7E2688B6822F0FB429C
:107BC00022F4800203F0F843134343F0E073E360D0
:107BD00040E7E36823F0FB4323F4800343F0C073E2
:107BE000E36037E7E2688B6822F0FB4222F4800210
:107BF00003F0F843134343F0A073E3602AE7E3681C
:107C000023F0FB4323F4800343F40003E36021E704
:107C100092FAA2F23AB1B2FA82F2012303FA02F224
:107C2000A0E70125EDE601229CE700BF0000C07D32
:107C3000FFFF170038B503689A68940702D59B6860
:107C4000002038BD9A68D1070ED59A6802F00D025F
:107C5000012A0BD0C36D43F01003C365036E43F0DC
:107C600001030366012038BD002038BD9A6822F068
:107C7000004222F03F0242F0020203219A601960A2
:107C8000044600F085F9236805469B68DB07EBD5C1
:107C900000F07EF9401B02282368F6D99A68D207C3
:107CA000F3D5E36D43F01003E365236E43F0010366
:107CB0002366012038BD00BF90F85830012B70B505
:107CC00057D003689A6801215207044680F858107B
:107CD00030D59A68DA68960104D5A18B40F201127A
:107CE000914261D09A68500702D59A6891074FD5A2
:107CF0009A68120740D40C2500F04AF9236806461A
:107D00009A68154219D000F043F9801B05282368B2
:107D1000F6D99A682A42F3D0E36D43F01003E36585
:107D2000236E43F0010323660125002384F85830B5
:107D3000284670BD9A681507CCD4DA68606D22F0C9
:107D40000102DA6090F82520022A3ED05A6822F01B
:107D500010025A602046FFF76DFF05460028E4D167
:107D6000E36D23F4885323F0010343F00103E3653B
:107D7000DBE70225284670BD9A689607BBD49A684F
:107D800022F0004222F03F0242F020029A60B2E765
:107D90009A6822F0004222F03F0242F010029A60FC
:107DA0009A681207A7D5E7E71A68550606D4184A55
:107DB00001E0013AB0D019684806FAD540221A60AD
:107DC0009A68510718D4042596E701F047F805464C
:107DD00060B1E36D226843F04003E365536823F02C
:107DE000100353602046FFF725FF9EE72268536883
:107DF00023F010035360ADE79A689207E3D49A68C2
:107E000022F0004222F03F0242F010029A60DAE7CC
:107E1000000040A3704700BF704700BF704700BF1D
:107E2000704700BF704700BF90F85820012A4BD020
:107E3000F0B504680E689DB0034600220120B4F13D
:107E4000A04F189283F85800199207D0D96D83F883
:107E5000582041F02001D9651DB0F0BD274DAA681A
:107E600052070AD5A268DA6D42F02002DA650120D5
:107E7000002283F858201DB0F0BDA06810F0040067
:107E8000F1D11EB3DFF878E04F68DEF8082093F8F0
:107E900038C022F460423A4342EA4C32CEF808201D
:107EA000A268D40727D4A86810F0010021D1DEF819
:107EB00008208C6822F4716121F00F0146EA040267
:107EC0000A43CEF80820D3E7022070470C4A916895
:107ED00021F460419160A068A968C90700F0010021
:107EE00007D430B9916821F4716121F00F019160DC
:107EF000BEE70020BCE7AA68BAE700BF0001005057
:107F00000003005038B50F4B1B680BB9012038BD7A
:107F10000D494FF47A720546B2FBF3F30868B0FBE3
:107F2000F3F001F03FF904460028EFD10F2DEDD812
:107F3000024629464FF0FF3001F0F0F8034B20468F
:107F40001D6038BD6C060020680600207006002009
:107F500000B5032083B001F0CFF80020FFF7D2FF77
:107F600018B1012003B05DF804FB0190FEF7E4FCBA
:107F7000019803B05DF804FB034A044913680968DB
:107F80000B441360704700BF407400206C06002053
:107F9000014B1868704700BF4074002038B5044694
:107FA000FFF7F6FF631C054602D0044B1B681C4418
:107FB000FFF7EEFF401BA042FAD338BD6C0600204D
:107FC000002800F06C812DE9F0410368D90782B0E8
:107FD00004462DD5B7498A68C96802F00C020C2AFC
:107FE00000F0F580082A00F0F7806368B3F5803F61
:107FF00000F02E81B3F5A02F00F0E081AD4D2A688E
:1080000022F480322A602A6822F480222A60002B1F
:1080100040F02381FFF7BCFF064605E0FFF7B8FFFD
:10802000801B642800F237812B689F03F6D42368F5
:108030009E0700F1A5801A0719D563699D4D002B95
:1080400000F0D780D5F8943043F00103C5F89430A0
:10805000FFF79EFF064605E0FFF79AFF801B022808
:1080600000F21981D5F894309F07F5D52368590798
:108070003FD5904B9A6DD20000F12B819A6D42F062
:1080800080529A659B6D03F080530193019B0126FA
:10809000894D2A68D70540F1EE80A368012B00F0D6
:1080A0001A81052B00F0CB81824DD5F8902022F06B
:1080B0000102C5F89020D5F8902022F00402C5F8FE
:1080C0009020002B40F00E81FFF762FF41F28837CD
:1080D000804606E0FFF75CFFA0EB0800B84200F224
:1080E000DA80D5F890309A07F4D4002E40F023813E
:1080F00023689B0618D5A3696E4D002B00F00781FD
:10810000D5F8983043F00103C5F89830FFF740FFE9
:10811000064605E0FFF73CFF801B022800F2BB800B
:10812000D5F898309F07F5D5E06928B3614DAA6866
:1081300002F00C020C2A00F04E812A68022822F07C
:1081400080722A6000F0FD80EA6822F00302EA6093
:10815000EA6822F0887222F48032EA60FFF718FFA2
:108160002C46054605E0FFF713FF401B022800F2EE
:10817000928023689B01F6D4002002B0BDE8F08114
:108180004C4A9368D26803F00C030C2B45D0042BA7
:1081900047D0E368474D002B00F083802B6843F401
:1081A00080732B60FFF7F4FE064604E0FFF7F0FE55
:1081B000801B02286FD82B685805F7D56B68226999
:1081C00023F0FE4343EA02636B60236833E701F068
:1081D000030103297FF409AF364A126892037FF541
:1081E00027AF6268002A7FF423AF012002B0BDE808
:1081F000F081D5F8943023F00103C5F89430FFF7EF
:10820000C7FE064604E0FFF7C3FE801B022842D8E3
:10821000D5F894309807F6D428E702F00302022A32
:10822000B7D1244B1B685D0502D5E368002BDCD079
:10823000204A20695368214923F0FE4343EA006342
:1082400053600868FFF75EFE0028CED12368F2E68F
:10825000184A136843F480331360FFF799FE154DF5
:10826000064604E0FFF794FE801B642813D82B68B1
:108270009B03F7D5DBE62A6842F480722A60FFF799
:1082800087FE07462B68D8053FF507AFFFF780FE4E
:10829000C01B0228F6D9032002B0BDE8F0810120FE
:1082A00070472B6823F480732B60FFF771FE06463E
:1082B0000BE000BF0010024000700040700600207C
:1082C000FFF766FE801B0228E5D82B685905F7D416
:1082D000BCE70026DCE6614AD2F8903043F00103A7
:1082E000C2F89030FFF754FE5C4D804641F288376B
:1082F00005E0FFF74DFEA0EB0800B842CBD8D5F85B
:1083000090309907F5D5002E3FF4F2AE13E0D5F882
:10831000983023F00103C5F89830FFF739FE064680
:1083200004E0FFF735FE801B0228B4D8D5F898305A
:108330009807F6D4F8E6494A936D23F08053936585
:10834000D6E6FFF725FE064604E0FFF721FE801B78
:108350000228A0D82B689901F7D4E968404B226A1B
:10836000A76AE66A606A0B401343D4E90C1243EA39
:108370000723013843EAC663490843EA0013013979
:10838000520843EA4153013A43EA4263EB602B68E7
:10839000324C43F080732B60EB6843F08073EB60EA
:1083A000FFF7F6FD054605E0FFF7F2FD401B02284A
:1083B0003FF671AF23689A01F6D5DDE603F18043FD
:1083C000A3F53C331A6842F480221A601A6842F41A
:1083D00080321A6041E701283FF408AFEB68226A57
:1083E00003F0030191427FF400AF616A03F0F002F1
:1083F0000139B2EB011F7FF4F8AEA16A03F4FE422B
:10840000B2EB012F7FF4F1AEE16A03F07842B2EBF8
:10841000C16F7FF4EAAE226B5208013A03F4C00147
:10842000B1EB425F7FF4E1AE626B5208013A03F0B8
:10843000C063B3EB426F14BF01200020D6E6074BA8
:10844000D3F8902042F00402C3F89020D3F8902093
:1084500042F00102C3F8902044E700BF0010024040
:108460000C809F01002800F00581AD4A2DE9F843FA
:10847000136803F00F038B420CD2136823F00F0331
:108480000B431360136803F00F038B4202D00120EB
:10849000BDE8F8830368DF0704460D4640F1888095
:1084A0004268032A00F0AD809E4B022A1B6800F050
:1084B000FF805B05EBD59B4B996801F00C0104290B
:1084C0000AD0996801F00C01082905D0996801F0DB
:1084D0000C010C2900F0FB804FF00008914EB368AE
:1084E00023F003031A43B260FFF752FD41F28837CD
:1084F000814605E0FFF74CFDA0EB0900B84274D8B7
:10850000B368626803F00C03B3EB820FF2D1236807
:108510009F0740F1D380580704D582498A6842F406
:10852000E0628A60190706D57E4A936823F47C537B
:1085300043F4E06393607B4AA168936823F0F003FF
:108540000B439360764E326802F00F02AA4237D88E
:1085500023685A0706D57349E0688A6822F4E06206
:1085600002438A601B0743D46E4A936803F00C03EE
:10857000042B00F0D380936803F00C03082B00F069
:108580009B80936803F00C030C2B75D00023654A85
:10859000654C9268654866490068C2F30312A25CA4
:1085A00002F01F02D3400B60BDE8F843FFF7AABCFE
:1085B0009E07B0D45A4E326802F00F02AA42C7D9C1
:1085C000326822F00F022A433260FFF7E1FC41F2E9
:1085D00088378046336803F00F03AB42B8D0FFF70B
:1085E000D7FCA0EB0800B842F4D90320BDE8F8831B
:1085F0004C4A2169936823F4605343EAC1039360B2
:10860000B2E74849086880017FF541AFCE68C86885
:10861000484F06F00306032ECE680CBF4649474973
:10862000C0F303100130B1FBF0F1C6F306203D4E5C
:1086300001FB00F1F068C0F3416001304000B1FB84
:10864000F0F1B9427FF648AFB16811F0F00F07D0F2
:1086500013F002083FF442AFA368002B7FF43CAF55
:1086600030498B6823F0F00343F080038B604FF0B8
:10867000800833E701207047D068D368D26800F0E3
:108680000300C3F303130328C2F3062203F101011D
:108690000CBF294B294BB3FBF1F303FB02F3214A37
:1086A000D268C2F3416201325200B3FBF2F36EE7CB
:1086B00099033FF500AFEAE61F4B68E7B8F1000FFA
:1086C0003FF440AFB36823F0F003B3603AE7D868F3
:1086D000D968184E00F003000328D8680CBF164B69
:1086E000164BC1F303110131B3FBF1F3C0F30621C3
:1086F0000C4803FB01F3C168C1F34161013149003A
:10870000B3FBF1F3B3427FF6E7AE836823F0F003E7
:1087100043F0800383604FF08008DFE6074B36E7C5
:108720000020024000100240B4B100087006002092
:108730006806002000B4C40400366E010024F40072
:10874000184B9A6802F00C02042A27D09A6802F0AB
:108750000C02082A24D09A6802F00C020C2A01D0DC
:1087600000207047D968D868DB6801F00301C0F3C6
:1087700003100329C3F3062300F101020CBF0A48CA
:108780000A48B0FBF2F000FB03F0064BDB68C3F3D2
:10879000416301335B00B0FBF3F07047034870475F
:1087A000014870470010024000366E010024F400BA
:1087B000014B1868704700BF68060020054B064A49
:1087C0009B680649C3F302230868D35C03F01F03C8
:1087D000D840704700100240C4B10008680600206D
:1087E000054B064A9B680649C3F3C2230868D35C5D
:1087F00003F01F03D840704700100240C4B10008C6
:10880000680600202DE9F0410368044613F40020B7
:1088100082B057D09F4B9A6DD00040F10D81002758
:108820009D4D2B6843F480732B60FFF7B1FB064628
:1088300005E0FFF7ADFB801B022800F20F812B68DB
:10884000D905F6D5934B216CD3F8902012F44072E1
:1088500028D08A4226D0D3F89000D3F8902042F452
:108860008032C3F89020D3F8902022F48032C3F8ED
:10887000902020F44075C207C3F8905012D51D46D1
:10888000FFF786FB41F28836804606E0FFF780FB63
:10889000A0EB0800B04200F2E180D5F890309B07D1
:1088A000F4D5216C7B4AD2F8903023F440730B430B
:1088B000C2F89030002027B1764A936D23F08053A0
:1088C00093652368DE0708D572496568D1F888206A
:1088D00022F003022A43C1F888209D0708D56D497C
:1088E000A568D1F8882022F00C022A43C1F888201C
:1088F000590708D56749E568D1F8882022F0300289
:108900002A43C1F888201A0708D562492569D1F899
:10891000882022F0C0022A43C1F888209F0608D58B
:108920005C496569D1F8882022F440622A43C1F885
:1089300088205E0608D55749A569D1F8882022F419
:1089400040522A43C1F888201D0608D55149E569DF
:10895000D1F8882022F440422A43C1F88820D90562
:1089600008D54C49256AD1F8882022F440322A43A0
:10897000C1F888209A0508D54649656AD1F888204B
:1089800022F440222A43C1F888205F050BD54149D3
:10899000A56AD1F8882022F440122A43B5F5801F39
:1089A000C1F888205CD01E050BD53A49E56AD1F89C
:1089B000882022F440022A43B5F5800FC1F88820B0
:1089C00053D0DD040BD53349256BD1F8882022F034
:1089D00040722A43B5F1807FC1F888204AD09904BB
:1089E0000BD52C49656BD1F8882022F040622A43D0
:1089F000B5F1006FC1F8882041D05A040BD5254944
:108A0000A56BD1F8882022F040622A43B5F1006FAF
:108A1000C1F8882038D01B040BD51E4AE16BD2F870
:108A2000883023F040530B43B1F1805FC2F88830A7
:108A30000DD002B0BDE8F0819A6D42F080529A6587
:108A40009B6D03F080530193019B0127E8E6D368F7
:108A500043F48033D36002B0BDE8F08103202AE7FD
:108A6000CA6842F48012CA609DE7CA6842F4801264
:108A7000CA60A6E7CA6842F48012CA60AFE7CA6853
:108A800042F48012CA60B8E7CA6842F48012CA6031
:108A9000C1E700BF00100240007000402DE9F04F18
:108AA000D1F800E083B0BEF1000F00F08180DFF864
:108AB000A09188460026012303FA06F212EA0E0767
:108AC00072D0D8E9011421F0100B06FA03FC0BF167
:108AD000FF35032303FA0CFA012D6FEA0A0A04FAA0
:108AE0000CF468D9C3680AEA03031C43C460026833
:108AF00001F0030302EA0A0A03FA0CF343EA0A0349
:108B0000CD00036050D54C4A136E43F00103136649
:108B1000136E26F0030404F1804403F0010304F50E
:108B20008034019306F00303019AA5689B000F228D
:108B30009A40B0F1904F25EA020213D03F4DA8426F
:108B40006BD03F4DA84263D03E4DA8426AD03E4D07
:108B5000A8426CD03D4DA8420CBF0525062505FA5C
:108B600003F31A43A260D9F80030FA43CC0354BF90
:108B700013403B43C9F80030D9F804308D0354BF8B
:108B800013403B43C9F80430D9F80830CC0254BF35
:108B900013403B43C9F80830D9F80C30890254BF60
:108BA00013403B43C9F80C3001363EFA06F382D13C
:108BB00003B0BDE8F08F8368D8F80C5003EA0A03CD
:108BC00005FA0CF51D4385604368C1F3001523EADF
:108BD00002032A46B2401A434260C36803EA0A030A
:108BE0001C43BBF1020FC46081D1F40800EB840484
:108BF00006F00703256AD8F810209B004FF00F0BF2
:108C00000BFA03FB25EA0B059A402A4322626EE722
:108C1000022505FA03F31A43A4E7012505FA03F335
:108C20001A439FE7032505FA03F31A439AE704253D
:108C300005FA03F31A4395E70010024000040048C8
:108C400000080048000C00480010004800140048CC
:108C5000000401400AB9816270478161704700BF1A
:108C6000436901EA030221EA030141EA0241816109
:108C7000704700BF00287CD003463F4A00689042FE
:108C80002DE9F04161D93D493D4A3E4C0144A2FBEA
:108C9000012109098900D3E902721E691C643A4363
:108CA0005C699D69DFF8F4E0DFF8CC8032434FF077
:108CB000020C224383F825C0314CD0F800C0DE6995
:108CC00059642A43C5B2083DA4FB05451C6A3243DA
:108CD0002CF4FF4C2C4E22432CF0700CC5F30414E2
:108CE000404598BF764642EA0C0289080125DFF824
:108CF000B0C0026005FA04F406EB810EB7F5804FB0
:108D00001C65C3E912EC29D05868C2B201380328A7
:108D100046F82120CCF8044026D81C491C48986508
:108D20001144013A890002F01F0205FA02F2002400
:108D30005965DA650C60426000200122D86383F82F
:108D4000240083F82520BDE8F08112490C4A124C1A
:108D50000144A2FB0121090989009CE700225A6015
:108D600046F82120CCF804400022C3E91522DA6538
:108D7000E2E70120704700BF07040240F8FBFDBF97
:108D8000CDCCCCCC00040240200802403F82001031
:108D900040090240F8FFFDBF000002400008024009
:108DA00080080240F0B490F82440012C4AD090F89A
:108DB00025400125AC4280F824503DD10468C76CA1
:108DC0000226002580F82560C5632668D0E914C511
:108DD00026F001062660C7F804C015B1D0E9166771
:108DE0007760466CD0F808C006F01F070126BE4029
:108DF000076C7E606360036BBCF1100F0BBFA26059
:108E0000A160E160E26003B3236843F00E032360D6
:108E1000836C1A68D20303D51A6842F480721A6010
:108E20001DB12B6843F480732B60236843F001036A
:108E300023600020F0BC7047002380F82430F0BC91
:108E4000022070470220F0BC7047236823F004031F
:108E50002360236843F00A032360D9E790F82520B4
:108E6000022A034609D00422C26301210022012004
:108E700083F8251083F824207047026870B4846C4E
:108E80001068DE6C20F00E00D3E9105110602068ED
:108E900020F4807020601468586D24F00104146080
:108EA00001F01F0101228A40196D6A60716038B1BA
:108EB0000268D3E9161422F48072026000204C602C
:108EC0000121002283F8251083F8242070BC70470C
:108ED00090F82530022B70B50AD00122042300211E
:108EE000C363144680F8252080F82410204670BD06
:108EF0000368856C1968C66C21F00E01D0E9104238
:108F00001960196821F0010119602B68416D23F483
:108F100080732B6002F01F0201239340026D636097
:108F2000726031B10B68D0E9162423F480730B60B2
:108F30005460836B0122002480F8252080F82440AF
:108F400013B19847204670BD1C46CFE770B4D0E9F6
:108F5000106304223168056803F01F039A400A4237
:108F60002C680AD014F0040F07D02B689B0637D565
:108F7000036B7260CBB170BC184702229A400A4260
:108F800015D014F0020F12D02B68990606D42B6866
:108F9000012123F00A032B6080F82510C36A726058
:108FA000002280F82420002BE5D170BC70470822F5
:108FB0009A400A42F9D02207F7D52A68416B22F07D
:108FC0000E022A60012202FA03F300247360C263D6
:108FD00080F8244080F825200029E6D070BC08479E
:108FE0002B6823F004032B60C2E700BF3B4A10B498
:108FF000136868B903F4C063B3F5806F14D0D2F876
:1090000080305DF8044B23F48073C2F880307047E1
:10901000B0F5007F2FD023F4C06343F48063136066
:1090200000205DF8044B7047D2F880102C4B2D487F
:1090300021F48071C2F88010116821F4C06141F4FC
:10904000007111601C685169322303FB04F3A0FB1B
:1090500003039B0C480503F1010306D500E023B18F
:109060005169490503F1FF33F9D41C4B5B695C0579
:10907000D6D50320D5E703F4C063B3F5806F09D0DC
:10908000D2F880305DF8044B43F480730020C2F8BE
:1090900080307047D2F88010114B124841F4807133
:1090A000C2F88010116821F4C06141F400711160B0
:1090B0001C685169322303FB04F3A0FB03039B0CE0
:1090C000480503F10103D0D501E0002BCDD0516953
:1090D000490503F1FF33C8D5F7E700BF0070004032
:1090E0006806002083DE1B43024A936843F48043F2
:1090F0009360704700700040074AD3684FF6FF0145
:109100000B40000243F0BF6300F4E06043F400331F
:109110000343D360704700BF00ED00E0184BDB68ED
:10912000C3F3022330B4C3F10705042D03F1040493
:1091300028BF0425062C19D9033B4FF0FF349C406F
:1091400022EA04044FF0FF32AA4021EA020101FAA8
:1091500003F2224312010028D2B20ADB00F1604080
:1091600000F5614080F8002330BC7047002423469E
:10917000E8E7044B00F00F0003441A7630BC704758
:1091800000ED00E0FCEC00E0002807DB044A00F002
:109190001F01012340098B4042F82030704700BF77
:1091A00000E100E00138B0F1807F0ED2084B10B42E
:1091B000084C5860F02084F8230000220721104654
:1091C0009A6019605DF8044B70470120704700BF3A
:1091D00010E000E000ED00E0B0B190F8213010B5F3
:1091E00003F0FF02044653B1002001236062C4E98A
:1091F0000100C4E90300606184F8213010BD80F8EB
:109200002020FDF7F3FBEFE70120704790F82130B5
:10921000012B05D0436A43F00203436201207047EB
:1092200070B40B688C694A680E6900682343134365
:10923000D1E902544A69016833431343044A2B437A
:1092400023430A401343036070BC0020704700BFF3
:1092500000F887FF88B1037910B503F0FF020446D8
:109260003BB10023022101222171184623612271A2
:1092700010BD4271FDF7D2FBF3E70120704700BF3C
:10928000F8B54379012B2DD00268022606710D46F0
:1092900004461168012005F0100700FA07F30B439C
:1092A00060711360FEF77AFE2268136865B903F0F7
:1092B0003E03B34203D1536843F0010353600123DB
:1092C000002023716071F8BDBE4003F47813B342EF
:1092D000F5D1536843F0020353600020012323714A
:1092E0006071F0E70220F8BD026838B501F01001A6
:1092F0000124136804FA01F1054623EA010120461E
:109300001160FEF74BFE2C71002038BDF8B5447992
:10931000069F012C60D004460D46266811460222A5
:1093200001202271607132685DBBA068DFF8C8C09F
:10933000C0F82CC0DFF8C4E0DFF8C4C042F48052AB
:10934000042FC0E90CEC326052D0082F4DD0002F12
:109350003CD00022376847F400573760FFF722FD02
:109360000023064663715EBB236801201A6805F07E
:10937000100500FA05F515431D60FEF70FFE304697
:10938000F8BDE068DFF87CC0C0F82CC0DFF878E0FA
:10939000DFF878C042F08052042FC0E90CEC326054
:1093A00020D0082F1BD0A7B10022376847F0005704
:1093B0003760FFF7F7FC002306466371002ED3D019
:1093C000236943F0040323613046F8BD06F1080227
:1093D000C0E706F11402E8E702263046F8BD06F1C0
:1093E0001C02E2E706F11802DFE706F11002B1E71E
:1093F00006F10C02AEE700BF7194000881940008EA
:1094000091940008799600088996000899960008BA
:10941000036870B501F0100204464FF480551868D7
:10942000954020EA050018601D68012000FA02F24C
:1094300025EA02020E461A60FEF7B0FD5EB1E06852
:10944000FFF70CFD2268136823F00053136001231B
:109450002371002070BDA068FFF700FD226813682B
:1094600023F40053136001232371002070BD00BF5B
:1094700010B5846A2046FBF701F80123237110BD63
:1094800008B5806AFAF7EEFF08BD00BF704700BF5D
:1094900010B5846A236943F0040323612046FFF773
:1094A000F5FF0123237110BD4379012B00F0888063
:1094B0002DE9F0418E68144602230122042E0D4648
:1094C0000746427103717FD0036804F01004EA6913
:1094D000012A6BD0D5E905C00721DA6BA14001282C
:1094E0006FEA010122F440485ED002286AD0BCFA3B
:1094F0008CF040094FF4807246EA0C06A24095F8C1
:1095000004C0064301EA0801D2436879BCF1010FA7
:1095100002EA01024FF40078296808BF46F4807619
:1095200008FA04F801286FEA080808BF46F4007634
:10953000022908EA020800F0828048EA0108A640F1
:1095400046EA0806DE631868D5E903124FF4804541
:10955000A54020EA05001860186840F6FE75A54091
:1095600020EA050501FA04F0284318601868C025B0
:10957000A54020EA050018609201186EC1F383012E
:1095800002F4706240F60F750A4305FA04F102FA1C
:1095900004F420EA01021443012100221C66104653
:1095A00039717A71BDE8F0810020A3E7996B2A6ACE
:1095B0001F20A04021EA0001A2400A439A6389E7E4
:1095C00002207047012095E7FEF7E2FC06462CB129
:1095D00014E0FEF7DDFC801B012839D83B685B6B8B
:1095E0001B04F6D40120FEF7D9FC3B686A6A1A64B2
:1095F0000EE0FEF7CDFC801B012829D83B685B6B91
:10960000002BF6DB0120FEF7C9FC3B686A6A5A644E
:1096100004F010049A6CA96AAE6840F2FF30A040D2
:1096200022EA0002A1400A439A64DA6CE96AFF2048
:10963000A04022EA0002A1400A43DA6447E7FFF7AC
:10964000B7F80B4B98420BD948F400483B6876E7D3
:109650003B69032243F008033B6110463A71A1E7DE
:10966000044A3B6890427FF66AAF48F4804866E758
:109670000068890900B4C40410B5846A2046FAF76A
:1096800019FF0123237110BD08B5806AFAF700FFA6
:1096900008BD00BF704700BF10B5846A236943F05E
:1096A000040323612046FFF7F5FF0123237110BD5A
:1096B000002800F08280F8B590F83D30044603F0B1
:1096C000FF0263B32268464EA569E0686168022321
:1096D00084F83D30B242136871D0B2F1804F52D05D
:1096E000A6F59436B2421FD006F58066B2421BD072
:1096F00006F59636B24217D006F54066B2426DD0F6
:1097000006F58066B24269D006F58066B24265D041
:1097100023F080032B431360D062916217E080F83E
:109720003C20FDF717FACDE7A6682E4F23F0700313
:109730003343266923F44073334323F080032B43E0
:10974000BA421360D06291622BD163691363012323
:109750005361002084F8483084F83E3084F83F306C
:1097600084F8403084F8413084F8423084F8433043
:1097700084F8443084F8453084F8463084F8473023
:1097800084F83D30F8BDA768266923F070033B4399
:1097900023F44073334323F080032B431360D062E0
:1097A0009162114B9A42D0D003F580639A42CCD09B
:1097B00003F580639A42CAD1C7E701207047A768C2
:1097C000266923F070033B4323F44073334323F0B3
:1097D00080032B431360D0629162B6E72669F3E7FA
:1097E000002C0140003401400040014090F83D3021
:1097F000012B01D0012070470368144A02219342D3
:1098000080F83D1018D0B3F1804F15D0A2F59432F6
:10981000934211D002F5806293420DD002F5963248
:10982000934209D002F54062934205D01A6842F093
:1098300001021A60002070479968054A0A40062A0A
:1098400002D0B2F5803FF1D100207047002C0140DA
:10985000070001000368196A41F21112114208D190
:10986000196A44F24442114203D11A6822F00102FB
:109870001A60012380F83D300020704790F83D3099
:10988000012B01D00120704703681649022280F89D
:109890003D20DA688B4242F00102DA6017D0B3F162
:1098A000804F14D0104A934211D002F58062934247
:1098B0000DD002F59632934209D002F540629342F0
:1098C00005D01A6842F001021A60002070479968BA
:1098D000064A0A40062A02D0B2F5803FF1D10020A4
:1098E000704700BF002C0140000400400700010049
:1098F00090F83C30012B00F0848002220368F0B421
:1099000080F83D209D680A68594C602A04EA0504E5
:109910004FF0010580F83C509C6074D01ED9554C26
:10992000A24200F08E8000F29680B2F5005F3ED039
:10993000B2F1101F00F08580702A2FD1D1E90152B9
:10994000CC6899682A4342EA042221F47F410A4301
:109950009A609A6842F077029A601FE0202A70D0DD
:109960006CD9402A33D0502A7FD11D6A1E6A4C68B8
:10997000CF6826F001061E629A6925F00A0122F0DE
:10998000F00242EA071221439A6119629A6822F4AE
:10999000401222F0700242F057029A600023012226
:1099A00080F83D2080F83C30F0BC18467047D1E983
:1099B0000152CC6899682A4342EA042221F47F418B
:1099C0000A439A609A6842F480429A60E6E71D6A08
:1099D0001E6A4C68CF6826F001061E629A6925F05F
:1099E0000A0122F0F00242EA071221439A61196249
:1099F0009A6822F4401222F0700242F047029A6004
:109A0000CCE7022070471C6A4D68CE6824F0100431
:109A10001C6299691A6A21F4704122F0A00242EA9C
:109A2000051241EA063199611A629A6822F44012DD
:109A300022F0700242F067029A60AFE70AB1102A82
:109A4000ACD1996821F4401142F0070221F0700175
:109A50000A439A60A2E708498A42F2D030318A422A
:109A6000EFD040398A4299D1EBE7302A96D1E8E726
:109A70008800CEFF2000100040001000704700BF9B
:109A8000704700BF704700BF704700BF03681A6986
:109A9000910710B5044603D5DA68920700F18A8071
:109AA0001A69520702D5DA68500770D41A6911078B
:109AB00002D5DA68120758D41A69D10602D5DA68D5
:109AC000D2063ED41A69D00703D5DA68D10700F16F
:109AD0008A801A69120603D5DA68100600F18B80B5
:109AE0001A69D10503D5DA68120600F18C801A696B
:109AF000500603D5DA68510600F18D801A69920686
:109B000003D5DA68900600F18E801A69D10203D578
:109B1000DA68D20200F18F801A69900203D5DA6800
:109B2000910200F190801A69520203D5DA6850025E
:109B300000F191801A69110202D5DA6812024AD442
:109B400010BD6FF010021A61DB69082213F4407F28
:109B50002277204640F09080FFF790FF2046FFF7E5
:109B600091FF002223682277ACE76FF008021A61A8
:109B7000DB6904229B07227720467AD1FFF77EFF1C
:109B80002046FFF77FFF00222368227794E76FF0DB
:109B900004021A619B69022213F4407F2277204657
:109BA00064D1FFF76BFF2046FFF76CFF00222368AC
:109BB00022777BE76FF002021A619B690122990705
:109BC000027750D1FFF75AFF2046FFF75BFF0022D4
:109BD0002368227764E76FF4000220461A61BDE82B
:109BE000104000F0ADB86FF001021A612046FAF79C
:109BF00073FC23686DE76FF080021A61204600F065
:109C000095F823686CE76FF480721A61204600F0C3
:109C10008FF823686BE76FF040021A612046FFF768
:109C200033FF23686AE76FF020021A61204600F0D4
:109C30007BF8236869E76FF480121A61204600F010
:109C400079F8236868E76FF400121A61204600F083
:109C500073F8236867E76FF480021A61204600F00A
:109C60006DF8236866E7FFF70BFFB0E7FFF708FF23
:109C70009CE7FFF705FF86E7FFF702FF71E700BFEC
:109C800090F83C30012B49D0F0B4254A05680F68A4
:109C9000022380F83D30012495426B6880F83C40F7
:109CA000AE6825D002F5006295422CD023F00073F7
:109CB00023F070033B43B5F1804F6B600AD0194B22
:109CC0009D4207D003F580639D4203D003F59C338A
:109CD0009D4204D18B6826F080061E43AE600023AF
:109CE000012280F83D2080F83C30F0BC18467047D7
:109CF0004C6823F47002224322F0007222F07002BA
:109D00003A436A60E6E74A6823F47004144324F097
:109D1000007424F070043C436C60DBE70220704761
:109D2000002C014000040040704700BF704700BF96
:109D3000704700BF704700BF704700BF704700BF4B
:109D4000704700BFD0F88830202B3CD100293CD090
:109D5000002A3AD090F88030012B34D030B44E4BEA
:109D60000468012580F880509C424FF00005C566CC
:109D700006D063681B0203D5236843F08063236029
:109D800083688165B3F5805F4FF00001A0F85C2027
:109D9000A0F85E200167456E19D0002B3CD1036905
:109DA000002B6CD07F23A0F8603022230021C0F864
:109DB0008C10C0F88830A368B5F1005F43F0010350
:109DC000A3603AD115E00220704701207047036973
:109DD000002B3ED02223C0F88C10C0F88830A36836
:109DE000FF2143F00103B5F1005FA0F86010A3600C
:109DF00023D1B0F8683093421FD8284B22680367FC
:109E000042F48072002380F880302260A26842F021
:109E100080521846A2601AE0B3F1805F33D022234B
:109E2000C0F88C10C0F88830A368A0F8601043F028
:109E30000103B5F1005FA360DBD0194B2268036713
:109E400042F49072002380F880301846226030BCC3
:109E500070472221C0F88C30C0F88810A36840F207
:109E6000FF1143F00103B5F1005FA0F86010A3609B
:109E700003D1B0F8683093420CD90A4BDEE7FF23D8
:109E8000A0F8603091E70369002B8BD03F23A0F846
:109E900060308AE7044BB1E700800040F9A3000876
:109EA00005A3000881A300085DA500082DE9F04185
:109EB000D0F88460202E32D1A1B39AB390F88040BC
:109EC000012C2CD00546806FA5F8562013464FF084
:109ED000000821220124C5F88C802965C5F884205A
:109EE000A5F8543085F880402A6868B1134FDFF830
:109EF00054C0C762124FC0F838802832C0E90CC77E
:109F0000FEF750FF88B92A68402313629368002047
:109F100043F0800385F880009360BDE8F081022063
:109F2000BDE8F0810120BDE8F0811023C5F88C3038
:109F300085F880802046C5F88460F1E74D9F0008D1
:109F40008D9F00087D9F0008704700BF08B503681B
:109F5000806A1B6813F020030BD10268A0F856300A
:109F6000936823F080039360136843F04003136009
:109F700008BDFFF7E9FF08BD704700BF08B5806A5C
:109F8000FFF7FAFF08BD00BF704700BF806A036893
:109F900010B5D0F88440D0F888109A68120601D520
:109FA000212C24D09A68520601D5222908D0D0F855
:109FB0008C3043F01003C0F88C30FFF7E5FF10BD84
:109FC0000022A0F85E201A6822F490721A609A6843
:109FD00022F0805222F001029A60C26E012A15D04E
:109FE00000232022C0F888200367C366DFE7002231
:109FF000A0F856201A6822F0C0021A609A6820243D
:10A0000022F400029A60C0F88440CBE71A6822F07C
:10A0100010021A60E4E700BF08B5836A0022A3F8C3
:10A020005E201846A3F85620FFF7AEFF08BD00BF1C
:10A03000704700BF0368DA6919682DE9F04140F6FE
:10A040000F052A42044698687BD0AB4D054000F0CE
:10A050009780D70709D5CE0507D501261E62D4F80B
:10A060008C6046F00106C4F88C60970702F0040685
:10A0700040F1D380C7070AD502271F62D4F88C703D
:10A0800047F00407C4F88C70002E40F0CC8017070E
:10A0900005D58E0600F1DF80002D40F0DC8015052F
:10A0A0000AD54F0108D54FF400651D62D4F88C50D5
:10A0B00045F02005C4F88C50D4F88C50002D70D099
:10A0C000960607D58D0640F1D380226F12B1204647
:10A0D00090472368D4F88C509968490603D415F04A
:10A0E000280500F0D6801A6822F490721A609A68E7
:10A0F00022F0805222F001029A60E26E012A03D11E
:10A100001A6822F010021A6000222021C4F8881078
:10A11000E266996822674A0640F1A6809A68E06F75
:10A1200022F040029A60002800F09E80734B836307
:10A13000FEF7CEFE002834D0E06FBDE8F041836B1F
:10A140001847970609D58E0605D5236F4BB32046D1
:10A15000BDE8F0411847C500F7D4E56E012D22D0C7
:10A16000D50201D547026ED4160610D50D0601D4CE
:10A1700000020CD5636FA3B12046BDE8F04118473B
:10A180005F4E3142E9D0D7077FF56FAF63E75706DF
:10A1900001D54E0670D415024ED4D30101D5002945
:10A1A0007DDBBDE8F081D706DAD5CE06D8D5102202
:10A1B0001A629A6812F0400276D0E06F01684A682D
:10A1C00092B2002AEDD0B4F85C509542E9D9A4F8D7
:10A1D0005E200A6812F0200217D1196821F48071FC
:10A1E0001960996821F0010199609968202521F092
:10A1F00040019960C4F88850E2661A6822F01002A3
:10A200001A60FEF72BFEB4F85C50B4F85E10691AC1
:10A2100089B22046FFF70CFFC3E7002E3FF437AFAB
:10A22000C6077FF534AF04261E62D4F88C6046F072
:10A230000206C4F88C602AE74800AED52046BDE887
:10A24000F04100F0AFBC4FF4801220461A62BDE826
:10A25000F04100F0A3BC08251D62D4F88C5045F0F5
:10A260000805C4F88C501AE72046FFF78DFE98E7E2
:10A27000C0007FF52FAF28E71A68202522F04002A2
:10A2800000211A602046C4F884506167FFF75CFE25
:10A2900087E72046FFF778FEC4F88C5081E7204618
:10A2A000BDE8F04100F07CBCB4F85E00B4F85E108C
:10A2B00089B280B200293FF474AFB4F85C10081A78
:10A2C00081B200293FF46DAF186820F490701860D7
:10A2D000986820F0805020F0010020259860C4F894
:10A2E0008850E2661868226720F010021A60204643
:10A2F000FFF79EFE55E700BF0100001019A00008FF
:10A3000020010004D0F888100268222938B504D052
:10A31000936943F00803936138BD526A90F8604036
:10A32000816D22400A70B0F85E20816D013A92B2D0
:10A33000A0F85E20B0F85E20013192B28165002A5B
:10A34000EAD10368196821F4907119609968202591
:10A3500021F001019960C0F88850C16E026701299F
:10A36000044604D0FAF7C4F80023E36638BD1A683F
:10A37000B0F85C1022F010021A60FFF759FEF3E704
:10A38000D0F888100268222938B504D0936943F0C8
:10A390000803936138BD516AB0F86050846D29405C
:10A3A00024F8021BB0F85E108465013989B2A0F868
:10A3B0005E10B0F85E1089B20029EBD1136823F467
:10A3C000907313609368202523F001039360C0F815
:10A3D0008850C36E0167012B044604D0FAF788F851
:10A3E0000023E36638BD1368B0F85C1023F0100357
:10A3F0001360FFF71DFEF3E72DE9F84F0368D969F5
:10A400001F689D68D0F88820222A05D09A6942F0FA
:10A4100008029A61BDE8F88FB0F86820002A00F0C1
:10A4200095808A0604467AD590F86060DFF8289116
:10A4300007F4807705F001054FF000084FF0040A9B
:10A440005B6AA26D33401370B4F85E302168A26D70
:10A45000013B9BB2A4F85E30D1F81CB001321BF076
:10A46000070FA2651DD01BF0010F08D03FB10123DB
:10A470000B62D4F88C3043F00103C4F88C301BF02D
:10A48000020F0BF004032AD045B102220A62D4F86D
:10A490008C2042F00402C4F88C2023BBD4F88C300A
:10A4A0006BBBB4F85E309BB2A3B92268116821F48B
:10A4B000807111609168202001EA09019160C4F85F
:10A4C0008800E16E236701291FD02046FAF710F8B3
:10A4D000C4F86C801BF0200F21D02368B0E7002B5C
:10A4E000DCD0002DDAD0C1F820A0D4F88C3043F0B5
:10A4F0000203C4F88C30D4F88C30002BD1D0204625
:10A50000FFF742FDC4F88C80CBE71368B4F85C1009
:10A5100023F0100313602046FFF78AFDD8E7B4F854
:10A520005E309BB2002B3FF475AFB4F868209A42BE
:10A530007FF670AF236807499A6822F080529A60CC
:10A540001A68216742F020021A6063E7B0F85E30B3
:10A5500060E700BF05A30008FEFFFFEF02682DE9DA
:10A56000F84FD16917689568D0F88830222B05D04C
:10A57000936943F008039361BDE8F88FB0F8683041
:10A58000002B00F093808B06044678D5B0F860600D
:10A59000DFF8249107F4807705F001054FF00008FB
:10A5A0004FF0040A536AA16D334021F8023BB4F81E
:10A5B0005E30A165013B9BB2A4F85E30D2F81CB0BE
:10A5C0001BF0070F1DD01BF0010F08D03FB1012376
:10A5D0001362D4F88C3043F00103C4F88C301BF0C4
:10A5E000020F0BF004032AD045B102211162D4F806
:10A5F0008C1041F00401C4F88C1023BBD4F88C30CB
:10A600006BBBB4F85E309BB2A3B92268116821F429
:10A61000807111609168202001EA09019160C4F8FD
:10A620008800E16E236701291FD02046F9F760FFFB
:10A63000C4F86C801BF0200F21D02268B2E7002BF9
:10A64000DCD0002DDAD0C2F820A0D4F88C3043F052
:10A650000203C4F88C30D4F88C30002BD1D02046C3
:10A66000FFF792FCC4F88C80CBE71368B4F85C1059
:10A6700023F0100313602046FFF7DAFCD8E7B4F8A4
:10A680005E309BB2002B3FF477AFB4F868209A425B
:10A690007FF672AF236807499A6822F080529A6069
:10A6A0001A68216742F020021A6065E7B0F85E3050
:10A6B00062E700BF81A30008FEFFFFEF836ADA07AD
:10A6C00010B406D50168C46A4A6822F400322243F5
:10A6D0004A609C0706D50168046B4A6822F4803200
:10A6E00022434A60590706D50168446B4A6822F440
:10A6F000802222434A601A0706D50168846B4A68A3
:10A7000022F4004222434A60DC0606D50168C46B8D
:10A710008A6822F4805222438A60990606D501682D
:10A72000046C8A6822F4005222438A605A0609D5D2
:10A730000168446C4A6822F480122243B4F5801FF9
:10A740004A600BD01B0606D50268C16C536823F41F
:10A7500000230B4353605DF8044B70474A68846CD8
:10A7600022F4C00222434A60ECE700BF002850D028
:10A77000D0F884302DE9F0410446002B44D0236802
:10A7800027696669BD492422C4F884201868A26834
:10A7900020F0010018601D68E0693A433243294007
:10A7A00002430A431A605A68E168B54EA769656AB0
:10A7B00022F440520A435A60B34299682BD0226A6D
:10A7C00021F06E4121F430613A430A439A60DA6A1B
:10A7D00006F5384622F00F022A43B342DA623AD035
:10A7E000A84A93425AD0A84A934200F03281A74A1D
:10A7F000934200F0E9804FF001120023A266C4E901
:10A800001C330120BDE8F08180F88030FCF7E8F9C6
:10A81000B5E70120704721F06E4121F430613943E2
:10A820009960DA6A9A4822F00F022A43DA62D0F875
:10A83000883003F44063B3F5806F00F0918140F2FB
:10A840005781B3F5006F00F0A181B3F5406FD2D10D
:10A850004FF4004054E18E4B8E4AD3F8883003F019
:10A860000303D35CB0F5004F00F01A81082BC2D867
:10A8700001A252F823F000BFC3A90008ADA8000848
:10A880006DAB0008F7A70008BDA90008F7A70008EE
:10A89000F7A70008F7A7000875AA00087C4B7E4AB6
:10A8A000D3F8883003F00C03D35CDBE7FDF798FFA7
:10A8B000002800F0C780656A6268784B33F815306D
:10A8C000B0FBF3F303EB5203B3FBF2F39BB2A3F140
:10A8D00010014FF6EF7291428DD82068C3600022BC
:10A8E000C4E91C224FF00111A166A36A002B40F0BD
:10A8F000A58023685A6822F490425A609A6822F030
:10A900002A029A601A68002142F001021A60C4F813
:10A910008C10FDF73DFB23681A68110706460ED41C
:10A920001A68500733D400232022C4F8842084F806
:10A930008030C4F888201846E366BDE8F081DD6900
:10A9400015F40015ECD1FDF723FB2368801BB0F153
:10A95000007F1A6880F0BC805207F0D5DA691705CD
:10A96000EDD54FF400621A621A6822F4D0721A60B0
:10A970009968202221F0010199600320C4F8842005
:10A9800084F88050C4F88820C4F88C20D5E7DD69AD
:10A9900015F48005C7D1FDF7FBFA2368801BB0F1E1
:10A9A000007F1A6880F094805107F0D5DA691205AB
:10A9B000EDD5D6E7B0F5004F00F0E080FDF7C0FE22
:10A9C00076E7FDF7FBFE73E7314BD3F8883003F0F1
:10A9D000C003402BEED026D9802B00F0C980C02BBD
:10A9E0007FF409AFB0F5004F4FF400407FF464AF3F
:10A9F00062682A49530831F81510B0FBF1F003EBF7
:10AA00004003B3FBF2F39AB2A2F110004FF6EF71DC
:10AA100088423FF6F0AE23F00F039BB2C2F342022E
:10AA2000206813435AE7002B7FF4E5AEB0F5004FE2
:10AA3000C7D1FDF7C3FE28B1656AD9E72046FFF705
:10AA40003DFE56E74FF001120023A266C4E91C3315
:10AA50004BE70F4BD3F8883003F03003102BA9D00D
:10AA6000E1D9202B00F08480302B7FF4C4AEB0F508
:10AA7000004FBDD04FF400401EE700BFF369FFCF89
:10AA8000008000400044004000480040004C00406E
:10AA900000100240CCB10008D0B10008E0B10008BD
:10AAA000082B3FF6A8AE01A252F823F033AA000803
:10AAB00067AB000883AB0008F7A700087DAB000870
:10AAC000F7A70008F7A70008F7A7000887AB00085A
:10AAD00022F4D0721A609A68202122F001029A6052
:10AAE0000320C4F8841084F88050C4F8881024E748
:10AAF000002B7FF480AEFDF761FE0028A2D0656ACE
:10AB00006668234B06EB460133F81520B0FBF2F3E1
:10AB10008B42FFF470AEB3EB063F3FF66CAE002500
:10AB200000232946F9F704FB0B0243EA10630202F3
:10AB30007008171843F1000832462B463846414644
:10AB4000F9F7F6FA134BA0F540729A423FF653AE6E
:10AB500022684FF00113D060C4E91C55A366C4E617
:10AB6000FDF7EEFDC9E7FDF73BFE64E70A48A3E603
:10AB7000B0F5004F08487FF49FAE39E7FDF7E0FDE0
:10AB800059E7054834E74FF4004031E70248B7E79A
:10AB9000E0B10008FFFC0F000024F400704700BF84
:10ABA000704700BF704700BF90F88020012A17D07F
:10ABB00030B402682421C0F8841003461068146879
:10ABC000002120F0005024F0010420251460596673
:10ABD00010600846C3F8845083F8801030BC70477A
:10ABE0000220704790F88020012A33D003462420A9
:10ABF0001A68F0B4C3F88400146810685D6E20F021
:10AC000001001060906820F06040014391607DB9C0
:10AC1000012108462025A3F868100021A3F86A0046
:10AC200014600846C3F8845083F88010F0BC704765
:10AC3000966895680848094FC6F342666D0F815DB6
:10AC4000405DBE5D7D5DC900C00091FBF6F190FBEB
:10AC5000F5F0DFE70220704700B20008F8B1000805
:10AC600090F88020012A33D0034624201A68F0B4DB
:10AC7000C3F88400146810685D6E20F00100106055
:10AC8000906820F06060014391607DB90121084621
:10AC90002025A3F868100021A3F86A001460084674
:10ACA000C3F8845083F88010F0BC704796689568AC
:10ACB0000848094FC6F342666D0F815D405DBE5D79
:10ACC0007D5DC900C00091FBF6F190FBF5F0DFE778
:10ACD0000220704700B20008F8B1000800285CD0DC
:10ACE00090F83A30052B58D090F83A30022B54D0D7
:10ACF0003A4B70B51A6E42F001021A661B6E82B0B2
:10AD000003F001030193019B90F83A3003F0FF0236
:10AD1000002B44D00446FBF7F5FEA36823F0200285
:10AD2000402A226841D06068E668116825690343BB
:10AD30003343E06A666A2B4321F010010143A56AA0
:10AD400011603343D4E90C602B432549156843EA6D
:10AD5000C64343EA0063207D2940012843EA0103FA
:10AD600014BF00214FF480710B4313609369002BD3
:10AD700009DBD4E90635206A91692B43034321F0AE
:10AD80003F010B43936194F83A3003F0FF004BB955
:10AD9000012384F83A3002B070BD0120704780F87A
:10ADA0003920B7E7002002B070BD666811682069DD
:10ADB000E56A3343034321F01001606A2943A56A21
:10ADC00011600343206B166805492B43656B43EA0A
:10ADD000C0433140207D43EA0563BEE700100240D6
:10ADE000113E00E040B190F83A20052A034603D016
:10ADF00090F83A20012A01D00120704701680A68C2
:10AE000010B442F0010204240A60002083F83A40A2
:10AE10005DF8044B704700BF60B190F83A20052AF6
:10AE2000034607D090F83A20022A03D090F83A203F
:10AE3000042A01D00120704701680A6810B422F08A
:10AE4000010201240A60002083F83A405DF8044BB7
:10AE5000704700BF0D4885460D480E490E4A002335
:10AE600002E0D458C4500433C4188C42F9D30B4ABE
:10AE70000B4C002301E013600432A242FBD3FBF72A
:10AE800005FFF5F701FAF9F745FCFEE70080002021
:10AE9000000000207406002060B200087406002044
:10AEA00048740020FEE70000F8B500BFF8BC08BCFD
:10AEB0009E467047F8B500BFF8BC08BC9E46704778
:10AEC000FB21F93FFB2109407CD91240FB211940AD
:10AED0007A6A1F407CD92240BBFD2540FB212940D6
:10AEE0003A462C407A6A2F405C4731407CD9324048
:10AEF0009C6B3440BBFD3540DB8F3740FB21394034
:10AF00001BB43A403A463C405AD83D407A6A3F40EA
:10AF10004C7E40405C4741406C1042407CD94240EE
:10AF20008CA243409C6B4440AC344540BBFD454043
:10AF3000CBC64640DB8F4740EB584840FB21494099
:10AF400083F9A200444E6E00FC291500D15727005A
:10AF5000DD34F50062DBC0003C9995004190430070
:10AF60006351FE00BBDEAB00B761C5003A6E240042
:10AF7000D24D42004906E00009EA2E001C92D100A1
:10AF8000EB1DFE0029B11C00E83EA700F53582004C
:10AF900044BB2E009CE98400B4267000417E5F0013
:10AFA000D6913900538339009CF439008B5F8400BB
:10AFB00028F9BD00F81F3B00DEFF97000F98050041
:10AFC000112FEF000A5A8B006D1F6D00CF7E3600E7
:10AFD00009CB2700464FB7009E663F002DEA5F0071
:10AFE000BA277500E5EBC7003D7BF100F739070094
:10AFF00092528A00FB6BEA001FB15F00085D8D0072
:10B00000300356007BFC4600F0AB6B0020BCCF0049
:10B0100036F49A00E3A91D005E619100081BE6006A
:10B0200085996500A0145F008D40680080D8FF00FE
:10B0300027734D0006063100CA561500C9A87300D3
:10B040007BE260006B8CC000020000000300000087
:10B05000040000000600000000000040FB21F93F52
:10B06000000000002D44743E000000809846F83C2B
:10B070000000006051CC783B00000080831BF03959
:10B080000000004020257A38000000802282E3364C
:10B09000000000001DF3693500000000000030438F
:10B0A00000000000000030C31B5B3630302C313014
:10B0B000710000001B5B25642C25647A00000000F1
:10B0C000256420252D313273000000001B5B3132D6
:10B0D000382C3235352C302C302C302C302C306341
:10B0E000000000001B5B3132392C3235352C3235F3
:10B0F000352C302C302C302C306300001B5B31336E
:10B10000302C3235352C3235352C3235352C302C2F
:10B11000302C3063000000001B5B3133312C3235A2
:10B12000352C3235352C3235352C3235352C302C0A
:10B13000306300001B5B3133322C3235352C323515
:10B14000352C3235352C3235352C3235352C3063B3
:10B15000000000001B5B3133332C3235352C323587
:10B16000352C3235352C3235352C3235352C3235BF
:10B17000356300001B5B2564730000001B5B3230ED
:10B18000302C3130307100001B5B25646200000000
:10B190000C0000003E00000025386C640000000038
:10B1A00025730000252A6C6400000000252A730026
:10B1B000070000000000000000000000010203047E
:10B1C0000607080900000000010203040104020848
:10B1D00000101010041010100210101008000000D1
:10B1E000010002000400060008000A000C00100024
:10B1F0002000400080000001080402040801010151
:10B200000101010307010000232D302B2000000065
:10B21000686C4C0065666745464700003031323344
:10B220003435363738394142434445460000000042
:10B2300030313233343536373839616263646566AC
:10B2400000000000706F77007371727400000000DE
:08B25000108FFF7F01000000D8
:04B25800690200087F
:04B25C0041020008A3
:10B2600004000020000000000000000000000000BA
:10B2700000000000000000000000000000000000CE
:10B2800000000000000000000000000000000000BE
:10B2900000000000000000000000000000000000AE
:10B2A000000000000000000000000000000000009E
:10B2B000000000000000000000000000000000008E
:10B2C0000000000001000000D03AFDFF0000000077
:10B2D00054183400000000002A04FFFE00000000A3
:10B2E000A9A5D00400000008A9A5D0040000000012
:10B2F0002A04FFFE00000000541834000000000083
:10B30000D03AFDFFD9D0EEFFA2D1EFFFBAB9F0FFDE
:10B31000C297F1FF5B7CF2FF037AF3FFF4A4F4FF22
:10B32000F512F6FF2EDBF7FFEE15FAFF75DCFCFFDA
:10B33000B1480000FE740400E37B0900C3770F00EE
:10B3400099821600AEB51E004929280067F4320024
:10B35000732C3F00FBE44C006E2F5C00DA1A6D008A
:10B36000ACB37F007B039400D310AA0006DFC100BA
:10B37000096EDB0052BAF600C0BC13018A6A3201C2
:10B3800038B55201A28A7401F7D49701D27ABC0170
:10B390004D5FE20128620902F15F310231325A0247
:10B3A000AEAF8302A2ACAD0208FBD702E66A02038D
:10B3B0009ECA2C0348E756030C8D80037E87A903A1
:10B3C00001A2D1032AA8F80320661E0400A94204A2
:10B3D000413F650412F98504BAA8A404EC22C10413
:10B3E000253FDB04F6D7F20451CB0705CEFA190549
:10B3F000E64B29052CA8350576FD3E05033E45059F
:10B400009B6048059B604805033E450576FD3E056B
:10B410002CA83505E64B2905CEFA190551CB0705B1
:10B42000F6D7F204253FDB04EC22C104BAA8A40439
:10B4300012F98504413F650400A9420420661E04F8
:10B440002AA8F80301A2D1037E87A9030C8D8003EB
:10B4500048E756039ECA2C03E66A020308FBD7029C
:10B46000A2ACAD02AEAF830231325A02F15F3102BB
:10B47000286209024D5FE201D27ABC01F7D497013C
:10B48000A28A740138B552018A6A3201C0BC130124
:10B4900052BAF600096EDB0006DFC100D310AA0025
:10B4A0007B039400ACB37F00DA1A6D006E2F5C0052
:10B4B000FBE44C00732C3F0067F43200492928005C
:10B4C000AEB51E0099821600C3770F00E37B09001A
:10B4D000FE740400B148000075DCFCFFEE15FAFFB5
:10B4E0002EDBF7FFF512F6FFF4A4F4FF037AF3FF67
:10B4F0005B7CF2FFC297F1FFBAB9F0FFA2D1EFFF78
:10B50000D9D0EEFF4681FEFFD01E05008FE20B0072
:10B51000A4A2120044231900D7101F00ACFD230081
:10B520003964270089AE2800D34227007F94220087
:10B530004F381A00C0F90D0053EFFDFF408BEAFFB2
:10B540000BA6D4FFC780BDFF62BDA6FF164C92FFBD
:10B55000014E82FF11EE78FF4E3278FFC5C881FFA1
:10B56000DBD396FF9DBAB7FF9901E4FFD2301A00F2
:10B5700098CA57004A5699009880DA005C51160123
:10B580007375470137996801A9CE7401FFF8670107
:10B590003B363F01F53EF90086B4960055561A0039
:10B5A0003C1889FFA115EAFE085F46FE52A2A8FDDD
:10B5B00057B01CFD3CE5AEFC047B6BFCE7CF5DFCAB
:10B5C00060AB8FFC708D08FDCD13CDFD987FDEFE46
:10B5D000F1643A00538BDA01FA02B5035E70BC05E0
:10B5E000918BE007FCCD0E0AF345330C1585390E1F
:10B5F0007E9C0D10B9189D111AEFD712CE4EB113C3
:10B600007B4920147B492014CE4EB1131AEFD71278
:10B61000B9189D117E9C0D101585390EF345330C1C
:10B62000FCCD0E0A918BE0075E70BC05FA02B503F3
:10B63000538BDA01F1643A00987FDEFECD13CDFD25
:10B64000708D08FD60AB8FFCE7CF5DFC047B6BFC6D
:10B650003CE5AEFC57B01CFD52A2A8FD085F46FEBB
:10B66000A115EAFE3C1889FF55561A0086B49600CB
:10B67000F53EF9003B363F01FFF86701A9CE7401A2
:10B6800037996801737547015C5116019880DA009B
:10B690004A56990098CA5700D2301A009901E4FF1F
:10B6A0009DBAB7FFDBD396FFC5C881FF4E3278FF46
:10B6B00011EE78FF014E82FF164C92FF62BDA6FF8D
:10B6C000C780BDFF0BA6D4FF408BEAFF53EFFDFF01
:10B6D000C0F90D004F381A007F942200D342270092
:10B6E00089AE280039642700ACFD2300D7101F0065
:10B6F00044231900A4A212008FE20B00D01E050003
:10B700004681FEFF20204672657175656E63790083
:10B710000000000B0100000064000000E8030000CE
:10B7200098AB020001000000C00F0020E54D0008AA
:10B730000D570008202020566F6C756D6520200085
:10B7400000000002020000000100000000000000F4
:10B750002000000000000000D0100020854E0008EE
:10B7600091560008202020204761696E202020008B
:10B7700000000001020300000100000001000000C1
:10B780000600000000000000F41A0020194600081E
:10B7900091560008204D6F64756C6174696F6E007E
:10B7A000000000030205000001000000000000008E
:10B7B0000300000001000000B80F0020454E000803
:10B7C000C956000820537175656C636820202000FD
:10B7D00000000002020A000001000000000000005A
:10B7E0002000000000000000DC120020854E000850
:10B7F000915600082046696C74657220434620000B
:10B800000000000403000000640000006400000069
:10B81000AC0D000000000000C40F0020214E000805
:10B82000915600082046696C7465722042572000CA
:10B830000000000403050000640000006400000034
:10B84000C409000000000000043D0020214E000853
:10B85000915600082046696C7465722051202000C2
:10B8600000000002030A00000100000001000000C7
:10B870002000000000000000EC120020214E000813
:10B88000915600082020205369676E616C202000CB
:10B89000000000080A000000010000000100000094
:10B8A000200000000000000028690020854E0008EC
:10B8B000DD57000809000000444300004C534200DB
:10B8C00055534200414D00000024F40001000000E7
:04B8D0001000000064
:040000050800AE55EC
:00000001FF
